:1000000016C3000033C3000031C300002FC300003B
:100010002DC300002BC3000029C3000027C300002C
:1000200025C3000023C3000021C300001FC300003C
:100030000C949B3E1BC3000019C3000017C30000B3
:1000400015C3000013C300000C94873E0FC30000CB
:100050000DC300000BC3000009C3000007C300006C
:1000600005C3000003C3000001C30000FFC200007D
:10007000FDC20000FBC20000F9C20000F7C2000090
:10008000F5C20000F3C20000F1C20000180A1D0A08
:100090002B0A300A350A3A0A3F0A440AD20DD70D14
:1000A000E50DEA0DEF0DF40DF90DFE0D4C124F129A
:1000B0005212551258125B125E126112991EBD1E29
:1000C000D01EE01EE31EF31E031F1C1FAE1EB11E3A
:1000D000131F161F191FB41EB71EBA1E0A24202490
:1000E00034244C24622478249C24B224C8249326EB
:1000F00000272D289828C029F52AE32BE12C192E5A
:100100006A2ED42E1F2F292F8A2FE52FE82FEB2FB1
:10011000EE2FF12FF42FF72FFA2FAC32C232D83254
:10012000EF3205331B33313347339B339E33A133D7
:10013000A433A733AA33AD33B03308348434003545
:1001400089351236893605376F37D9375238BF3877
:100150003639BC393F3A00000000000000000404BA
:100160000404000400000A0A0A00000000000A0A51
:100170001F0A1F0A0A00040F140E051E0400181996
:100180000204081303000C12140814120D000C04CE
:100190000800000000000204080808040200080427
:1001A0000202020408000004150E150400000004F9
:1001B000041F04040000000000000C0408000000FC
:1001C000001F0000000000000000000C0C000001F7
:1001D0000204081000000E11131519110E00040C72
:1001E000040404040E000E11010204081F001F0283
:1001F000040201110E0002060A121F0202001F1063
:100200001E0101110E000608101E11110E001F0123
:100210000204080808000E11110E11110E000E1133
:10022000110F01020C000001020408100000000C74
:100230000C000C040800020408100804020000006E
:100240001F001F00000008040201020408000E1134
:100250000102040004000E11010D15150E000E110F
:1002600011111F1111001E11111E11111E000E116E
:10027000101010110E001C12111111121C001F1071
:10028000101E10101F001F10101E101010000E1155
:10029000101711110E001111111F111111000E0470
:1002A000040404040E000702020202120C001112E0
:1002B0001418141211001010101010101F00111B30
:1002C00015151111110011111915131111000E112D
:1002D000111111110E001E11111E101010000E111F
:1002E000111115120D001E11111E141211000F1004
:1002F000100E01011E001F04040404040400111167
:10030000111111110E0011111111110A0400111116
:10031000111115150E0011110A040A111100111105
:10032000110A040404001F01020408101F000E0833
:10033000080808080E00110A1F041F0404000E021A
:10034000020202020E00040A110000000000000078
:10035000000000001F000804000000000000000072
:100360000E010F110F0010101E1111111E000000C0
:100370000E1010110E0001010D1311110F000000DD
:100380000E111F100E000609081C08080800000FB7
:1003900011110F010E001010161911111100040097
:1003A0000C0404040E000200060202120C001010DD
:1003B0001214181412001808080808081C0000007D
:1003C0001A15151111000000161911111100000065
:1003D0000E1111110E0000001E111E101000000061
:1003E0000F110F010100000016191010100000007D
:1003F0000E100E011E0008081C0808090600000067
:10040000111111130D0000001111110A0400000058
:10041000111111150A000000110A040A1100000050
:1004200011110F010E0000001F0204081F003844C4
:1004300044447C4444007C40407844447800784400
:100440004478444478007C404040404040000C14D4
:10045000242424243C447C40407840407C00545474
:100460005438545454003844041804443800444464
:100470004C546444440054444C5464444400444840
:100480005060504844001C24242424246400446CFC
:100490005454444444004444447C44444400384458
:1004A0004444444438007C44444444444400784434
:1004B00044784040400038444040404438007C107C
:1004C0001010101010004444443C044438003854C8
:1004D0005454381010004444281028444400444424
:1004E000444444447E02444444443C040400545480
:1004F000545454547C005454545454547E02602038
:100500002038242438004444446454546400404057
:100510004078444478003844041C0444380048546B
:100520005474545448003C44443C14244400000097
:1005300038043C443C0000007840784478000000D7
:10054000784C784C78000000784040404000000033
:10055000182828287C44000038447C403C000000D7
:1005600054543854540000007804380478000000D3
:10057000444C546444000010444C54644400000053
:1005800044487048440000001C24444444000000D7
:10059000446C545444000000484878484800000027
:1005A0003844444438000000784848484800000077
:1005B0007048704040000000384040403800000063
:1005C0007C1010101000000048483808700000002F
:1005D000385454381000000044281028440000000B
:1005E000484848487C040000484838080800000093
:1005F000545454547C000000545454547E0200005F
:1006000060203C223C0000004242724A720000001E
:1006100040407844780000007008780870000000BE
:100620004C5272524C0000003C443C4444001124A3
:100630001FBECFEFD0E1DEBFCDBF15E0A0E0B1E03F
:10064000E4E5F9E800E00BBF02C007900D92A43D7D
:10065000B107D9F726E0A4EDB5E001C01D92A4389A
:10066000B207E1F70E94F93E0C94A844C9CCE2E637
:10067000F0E090819E7F9083908194609083908140
:10068000977F9083A8988BBB8DE08A95F1F7000047
:10069000A89A8081886080830895E2E6F0E09081E6
:1006A000916090839081946090839081977F9083F4
:1006B000A8988BBB8DE08A95F1F70000A89A8081FD
:1006C000886080830895CF93C82F892FE6DF8C2F11
:1006D000CF91E3CFE2E6F0E020812160208320810A
:1006E000246020832081277F2083A8988BBB92BB26
:1006F0008DE08A95F1F70000A89A80818860808358
:100700000895CF93C82F86E3B2DFC13049F030F0AF
:10071000C23041F0C33059F488EE07C088E403C00A
:1007200088E203C088E8B9DF04C0B7DF0BC0CD7F23
:1007300049F48FEE90E09093D7058093D6058FE330
:1007400091E008C08FE391E09093D7058093D605A0
:100750008FEE90E09093D5058093D405CF910895C6
:10076000CF93C82F8FEF8ABB81BB8093610081E05C
:1007700084BBE2E6F0E080818260808381E077DF05
:100780002FEF89E698E1215080409040E1F700C0CA
:10079000000080EC6CDF85E280DF81EC68DF81E1C6
:1007A0007CDF85EC64DF8BE278DF8BE276DF87EC41
:1007B0005EDF86E872DF8C2FA4DF8AE358DF85E0F6
:1007C0006CDF81EB54DF80E068DF88E166DF86EB79
:1007D0004EDF8AE062DF82E860DF87E25EDF81E190
:1007E00046DF2FEF8DEE92E0215080409040E1F700
:1007F00000C0000089E2CF913ACF0F931F93CF93AF
:10080000DF938C01EB018AE232DFC8015CDFCE01AD
:10081000DF91CF911F910F9156CF0F931F93CF93DD
:10082000DF938C01EB018BE222DFC8014CDFCE01AC
:10083000DF91CF911F910F9146CFCF93DF93EB01C3
:10084000BC01DBDFBE01CE01E8DF8CE2DF91CF919E
:100850000ECFCF93DF93EA01F0DFCE01DF91CF918E
:1008600039CF8F929F92AF92BF92CF92DF92EF9249
:10087000FF920F931F93CF93DF93A8956817790783
:1008800038F4862797276827792786279727A895FA
:100890002417350738F442275327242735274227C2
:1008A0005327A895A091D605B091D705FC01A817AC
:1008B000B90708F4FD016B01A617B70708F46D012D
:1008C0008091D4059091D505EA018417950708F425
:1008D000EC0179018217930708F47C01A895960131
:1008E0002F5F3F4F2E1B3F0BD7011196AC1BBD0B4B
:1008F0000E9470414B015C01B601CF017EDFA895DB
:10090000B701CE018ADF8CE2B2DEA895C12CD12CD2
:100910007601C814D904EA04FB0449F0C801DADE00
:10092000A8958FEFC81AD80AE80AF80AF2CFDF9123
:10093000CF911F910F91FF90EF90DF90CF90BF90DC
:10094000AF909F908F9008950F931F93411551057D
:1009500079F02115310561F0FA01AB01615071099F
:10096000260F371FBC01615071096E0F7F1F79DFA1
:100970001F910F9108952F923F924F925F926F9225
:100980007F928F929F92AF92BF92CF92DF92EF921F
:10099000FF920F931F93CF93DF93CDB7DEB7679787
:1009A0000FB6F894DEBF0FBECDBF5C01798B688BAC
:1009B000598748873B872A870F83F12C28E0029FBD
:1009C000C00111241A821982E8E0F0E0FF8BEE8B5F
:1009D00047019C01285F31093B8B2A8BFC01E052C7
:1009E000F340FD8BEC8BC888D98889819A81C80E29
:1009F000D91E8A899B89EE89FF898E1B9F0B9C01DA
:100A00002A5A3E4F3F872E878C899D898E1B9F0BCC
:100A1000FC01EA5AFE4FFD87EC871E821D821C8274
:100A20001B8287E0682E712C412C512C212C312CFB
:100A3000FF81F7FD1EC0EE85FF85849190E0062CB6
:100A400002C0959587950A94E2F780FF08C0088553
:100A500019859701A701B6018D819E8107C00A857E
:100A60001B859701A701B6018B819C818A0D9B1D77
:100A700020C0FF81F03CF0F0EC85FD85849190E092
:100A8000062C02C0959587950A94E2F780FF09C06D
:100A9000088519859701A701B601C501820D931D2F
:100AA00008C00A851B859701A701B601C501840D01
:100AB000951D4ADF280C391C480C591CF1E06F1AAF
:100AC00071082B813C81280D391D3C832B838D813E
:100AD0009E81880D991D9E838D839FEF69167906EF
:100AE00009F0A6CFEE89FF893197FF8BEE8B298124
:100AF0003A812E0D3F1D3A832983EF2B09F073CFE6
:100B000067960FB6F894DEBF0FBECDBFDF91CF91D1
:100B10001F910F91FF90EF90DF90CF90BF90AF901B
:100B20009F908F907F906F905F904F903F902F900D
:100B300008954F925F926F927F928F929F92AF92A1
:100B4000BF92CF92DF92EF92FF920F931F93CF93BA
:100B5000DF93EC016B014A013901102F88E0089FF7
:100B6000500111242701F20101912F010023B1F05E
:100B70002091D6053091D705CE0108962817390760
:100B800020F4CA0CDB1CC1E0D0E0E12E9301A401EB
:100B9000B601CE01F0DECA0DDB1DE5CFDF91CF91AE
:100BA0001F910F91FF90EF90DF90CF90BF90AF908B
:100BB0009F908F907F906F905F904F9008956F926D
:100BC0007F928F929F92AF92BF92CF92DF92EF92DD
:100BD000FF920F93CF93DF9300D000D0CDB7DEB755
:100BE0006C015B014A013901C70119821A821B821B
:100BF0001C824AE0BE016F5F7F4F0E947F41CE01A1
:100C000001967C019301A401B501C60192DF0F900A
:100C10000F900F900F90DF91CF910F91FF90EF9079
:100C2000DF90CF90BF90AF909F908F907F906F900C
:100C300008950F931F932091D4053091D5056091AD
:100C4000D6057091D7058C0140E050E080E090E03F
:100C500008DE1F910F910895EF92FF920F931F935B
:100C6000CF93DF93EB018A017901BC01640F751FFB
:100C7000C4DDBE01CE01D1DD8CE2F9DCC0E0D0E004
:100C8000C017D10721F0C70125DD2196F9CFDF91EB
:100C9000CF911F910F91FF90EF900895EF92FF92E7
:100CA0000F931F93CF93DF93EB018A017901BC016E
:100CB000A4DDBE01600F711FCE01AFDD8CE2D7DC79
:100CC000C0E0D0E0C017D10721F0C70103DD2196B5
:100CD000F9CFDF91CF911F910F91FF90EF90089581
:100CE0002F923F924F925F926F927F928F929F923C
:100CF000AF92BF92CF92DF92EF92FF920F931F932A
:100D0000CF93DF9300D000D000D0CDB7DEB76C0119
:100D10007B015A0139012801261B370B3A832983AD
:100D20008A01081B190B17FF03C0119501951109C2
:100D3000CA14DB0420F022242A94322C03C022247B
:100D40002394312C89819A819E838D8397FF05C0DE
:100D50009195819591099E838D832D813E81319559
:100D6000219531093C832B83E614F70428F08FEF9B
:100D70009FEF9A83898304C021E030E03A8329837E
:100D800048018D819E81881A990AA201B701C60186
:100D900060DDC401880F991F2B813C818217930766
:100DA00064F0CA14DB0499F02D813E81821A930A03
:100DB000C20CD31C0817190744F3E614F70439F0E2
:100DC000800E911E89819A81E80EF91EDECF26964B
:100DD0000FB6F894DEBF0FBECDBFDF91CF911F914C
:100DE0000F91FF90EF90DF90CF90BF90AF909F90CA
:100DF0008F907F906F905F904F903F902F900895CD
:100E0000AF92BF92CF92DF92EF92FF920F931F9318
:100E1000CF93DF937C016B01EA01590198011CDF3C
:100E2000B501615071096C0D7D1D9801AE01C701BE
:100E300013DF9801A501B601C70130DFCE0101978C
:100E40009801A501B6018E0D9F1DDF91CF911F91D5
:100E50000F91FF90EF90DF90CF90BF90AF901ECF9B
:100E60002F923F924F925F926F927F928F929F92BA
:100E7000AF92BF92CF92DF92EF92FF920F931F93A8
:100E8000CF93DF931C012B01690150E0002711274C
:100E9000041B150BC1E0D0E0C41BD50BCC0FDD1F2C
:100EA000E12CF12CA6015701A40CB51CB5013101B0
:100EB000601A710AC301CDDCA601B5014801820C9C
:100EC000931CC401C6DCA6015201AE18BF08B501CF
:100ED000C401BFDCA601B501C301BBDCEC16FD06F5
:100EE000B4F08FEFE81AF80AC701880F991F01962E
:100EF0008C0F9D1F22273327201B310BE216F30690
:100F000039F40C171D074CF0C0E0D0E001C0CE0151
:100F10000C171D0714F0EC01C5CF0F5F1F4F980190
:100F2000220F331F2F5F3F4F820F931F10161106A2
:100F300094F7DF91CF911F910F91FF90EF90DF9089
:100F4000CF90BF90AF909F908F907F906F905F9069
:100F50004F903F902F9008954F925F926F927F92A3
:100F60008F929F92AF92BF92CF92DF92EF92FF92B9
:100F70000F931F93CF93DF93EC015B014A0139017B
:100F800028018601ADDE9701A201B301C401A8DEEC
:100F90009501AE01B701C201A3DEDF91CF911F9190
:100FA0000F91FF90EF90DF90CF90BF90AF909F9008
:100FB0008F907F906F905F904F900895CF93C82F40
:100FC0008A3011F48DE0FADF5D9BFECFCCB980E072
:100FD00090E0CF910895CF92DF92EF92FF920F931E
:100FE0001F93A8950FEF1FEF21E430E04FE550E08D
:100FF00065E070E085E090E003DFA89521E430E053
:101000004FE550E06BE470E085E090E0F9DE2BE422
:1010100030E04FE550E061E970E085E090E0F0DE1F
:10102000A2E2EA2EA5E0FA2E01E02FE130E04FEF38
:101030005FEF60E570E082E190E07BDDBDE1EB2EEB
:10104000B5E0FB2E2FE130E04FEF5FEF6AE570E097
:1010500083E290E06EDD0FEF1FEF21E430E04FE51B
:1010600050E065E070E08CED90E0CADE21E430E015
:101070004FE550E06BE470E08CED90E0C1DE2BE4D6
:1010800030E04FE550E061E970E08CED90E0B8DED3
:1010900012E2E12E15E0F12E01E02FE130E04FEFFA
:1010A0005FEF60E570E08BEE90E043DD87E1E82ED6
:1010B00085E0F82E2FE130E04FEF5FEF6AE570E05A
:1010C0008CEF90E036DD99E4E92E92E0F92E2FE1E5
:1010D00030E04FEF5FEF66EE70E08AE090E029DDF0
:1010E000A8958091100690911106019709F04FC0C4
:1010F0000FE110E024E430E048E550E064E970E0FE
:1011000088E090E021DC2CE430E04EE650E06CE832
:1011100070E089E690E018DC24E430E048E550E037
:1011200064E970E080EE90E00FDC20EE37E048E20A
:1011300064EB70E080EA90E093DE20EE37E047E277
:1011400064EB70E080EA90E08BDE20EE37E04BE26B
:1011500064EB70E080EA90E083DE20EE37E045E269
:1011600064EB70E080EA90E07BDEE0EECE2EE7E01C
:10117000DE2EF4EBEF2EF12C07EB10E028EC30E044
:1011800044E950E060EA70E084E990E0E5DEA8958B
:101190008091100690911106892B09F051C00FE142
:1011A00010E024E430E048E550E064E970E088E0D5
:1011B00090E0CADB2CE430E04EE650E06CE870E0F2
:1011C00089E690E0C1DB24E430E048E550E064E9E2
:1011D00070E080EE90E0B8DB20E038EF48E264EBAE
:1011E00070E080EA90E03CDE20E038EF47E264EB1C
:1011F00070E080EA90E034DE20E038EF4BE264EB10
:1012000070E080EA90E02CDE20E038EF45E264EB0D
:1012100070E080EA90E024DE00E018EF23E230E0A6
:1012200045E050E065EA70E086E990E08DDB23E27E
:1012300030E045E050E065EA70E085EA90E084DB6C
:10124000A8958091120690911306892B79F4A895A0
:101250007DE0E72E75E0F72E01E02FE130E04FEF63
:101260005FEF63E270E08AE090E063DC8091120659
:10127000909113060197E1F4A89556ECE52E55E000
:10128000F52E01E02FE130E04FEF5FEF64E170E019
:1012900084E190E04EDC60ECE62E65E0F62E2FE176
:1012A00030E04FEF5FEF68E270E08EE190E041DC0C
:1012B000A89580911206909113060297E1F4A895E3
:1012C00039EBE32E35E0F32E01E02FE130E04FEF74
:1012D0005FEF64E170E084E190E02BDC40ECE42E11
:1012E00045E0F42E2FE130E04FEF5FEF68E270E071
:1012F0008EE190E01EDCA895809112069091130675
:10130000039779F4A89522EBE22E25E0F22E01E076
:101310002FE130E04FEF5FEF63E270E089E190E0B2
:1013200008DCA8958091120690911306049779F431
:10133000A89593EDE92E94E0F92E01E02FE130E03D
:101340004FEF5FEF63E270E08FE090E0F2DBA89593
:1013500080911206909113060597E1F4A8950DEC83
:10136000E02E04E0F02E01E02FE130E04FEF5FEFE0
:1013700064E170E089E190E0DCDB83ECE82E84E05E
:10138000F82E2FE130E04FEF5FEF63E270E08FE087
:1013900090E0CFDBA89580911206909113060697F6
:1013A000E1F4A895BDECEB2EB4E0FB2E01E02FE1BB
:1013B00030E04FEF5FEF64E170E089E190E0B9DB8E
:1013C00011EBE12E14E0F12E2FE130E04FEF5FEF53
:1013D00063E270E08FE190E0ACDBA89580911206AB
:1013E00090911306079779F4A895A8E9EA2EA4E04E
:1013F000FA2E01E02FE130E04FEF5FEF63E270E0A3
:101400008FE090E096DB8091120690911306892B75
:1014100009F048C0A895E0916F068E2F90E08830C3
:10142000910508F03FC0FC01EA5BFF4F0C94674157
:10143000F3E9EF2EF4E0FF2E04C0EEE8EE2EE4E038
:10144000FE2E02E02FE130E04FEF5FEF6EE170E043
:101450008BEE90E026C074E8E72E74E0F72E18C0FB
:101460006AE7E62E64E0F62E13C050E7E52E54E05E
:10147000F52E0EC046E6E42E44E0F42E09C03CE50D
:10148000E32E34E0F32E04C022E5E22E24E0F22E17
:1014900001E02FE130E04FEF5FEF6EE170E086EEAC
:1014A00090E047DB8091120690911306019701F5B9
:1014B000A89580911B06813069F038F08230C1F424
:1014C00000E7E02E04E0F02E09C094E8E92E94E055
:1014D000F92E04C08AE7E82E84E0F82E01E02FE11F
:1014E00030E04FEF5FEF6EE170E086EE90E021DBE1
:1014F0008091120690911306029701F5A8958091AC
:101500002206813069F038F08230C1F4A0E7EA2E7B
:10151000A4E0FA2E09C014E8E12E14E0F12E04C074
:10152000BAE7EB2EB4E0FB2E01E02FE130E04FEF05
:101530005FEF6EE170E086EE90E0FBDA80911206DC
:1015400090911306039779F4A895FEEDEF2EF4E041
:10155000FF2E01E02FE130E04FEF5FEF6EE170E032
:101560008EEE90E0E6DA80911206909113060497D1
:1015700001F5A89580917A06813069F038F08230C3
:10158000C1F460E7E62E64E0F62E09C0E4E8EE2E32
:10159000E4E0FE2E04C07AE7E72E74E0F72E01E0C7
:1015A0002FE130E04FEF5FEF6EE170E086EE90E00C
:1015B000C0DA8091120690911306059701F5A8955F
:1015C00080916E06813069F038F08230C1F430E7E6
:1015D000E32E34E0F32E09C054E8E52E54E0F52E56
:1015E00004C04AE7E42E44E0F42E01E02FE130E0AD
:1015F0004FEF5FEF6EE170E086EE90E09ADA809157
:10160000120690911306069701F5A89580916B0636
:10161000813069F038F08230C1F480E7E82E84E050
:10162000F82E09C024E8E22E24E0F22E04C09AE746
:10163000E92E94E0F92E01E02FE130E04FEF5FEF6B
:101640006EE170E086EE90E074DA8091120690917F
:101650001306079709F4A8951F910F91FF90EF903B
:10166000DF90CF900895CF92DF92EF92FF920F9389
:101670001F93A89500EE17E021E430E048EC50E01D
:101680006AEA70E085E090E05FD90FEF1FEF21E498
:1016900030E048EC50E063E270E085E090E0B0DBE1
:1016A00086E6E82E82E0F82E01E02FE130E040EE01
:1016B00057E06CE370E088E290E03BDA0FEF1FEF59
:1016C00020E530E040E550E065E070E08BEE90E032
:1016D00097DB90EEC92E97E0D92E24E1E22EF12C73
:1016E00003E111E026E430E041E351E066E470E01C
:1016F00085EF90E031DC37E1E32EF12C24E430E09B
:101700004FE251E064E470E087EF90E025DC0FEFFA
:101710001FEF20E530E040E550E064E670E08BEE3E
:1017200090E06EDB45EAE42EF12C03E111E023E7C3
:1017300030E041E351E063E770E085EF90E00CDCDE
:1017400053EAE52EF12C25E730E04FE251E065E762
:1017500070E087EF90E000DC65E3E62E65E0F62EB2
:1017600002E020EE37E040E050E068EC70E08DE20F
:1017700090E0DFD91F910F91FF90EF90DF90CF9015
:101780000895CF92DF92EF92FF920F931F93A89547
:1017900000EE17E021E430E048EC50E06AEA70E047
:1017A00085E090E0D1D80FEF1FEF21E430E048EC66
:1017B00050E063E270E085E090E022DB82EAE82E10
:1017C00084E0F82E01E02FE130E040EE57E06CE3DA
:1017D00070E088E290E0ADD90FEF1FEF20E530E038
:1017E00040E550E065E070E08BEE90E009DB90EEC4
:1017F000C92E97E0D92E24E1E22EF12C03E111E06D
:1018000026E430E041E351E066E470E085EF90E0EB
:10181000A3DB37E1E32EF12C24E430E04FE251E08A
:1018200064E470E087EF90E097DB0FEF1FEF20E5B7
:1018300030E040E550E064E670E08BEE90E0E0DA06
:1018400045EAE42EF12C03E111E023E730E041E327
:1018500051E063E770E085EF90E07EDB53EAE52E30
:10186000F12C25E730E04FE251E065E770E087EFCB
:1018700090E072DB6EECE62E65E0F62E02E020EEE4
:1018800037E040E050E068EC70E08DE290E051D944
:101890001F910F91FF90EF90DF90CF900895CF921E
:1018A000DF92EF92FF920F931F93A89500EE17E03F
:1018B00021E430E048EC50E06AEA70E085E090E036
:1018C00043D80FEF1FEF21E430E048EC50E063E233
:1018D00070E085E090E094DA81E4E82E84E0F82E70
:1018E00001E02FE130E040EE57E06CE370E088E289
:1018F00090E01FD90FEF1FEF20E530E040E550E00A
:1019000065E070E08BEE90E07BDA90EEC92E97E018
:10191000D92E24E1E22EF12C03E111E026E430E09F
:1019200041E351E066E470E085EF90E015DB37E1DC
:10193000E32EF12C24E430E04FE251E064E470E067
:1019400087EF90E009DB0FEF1FEF20E530E040E587
:1019500050E064E670E08BEE90E052DA45EAE42E67
:10196000F12C03E111E023E730E041E351E063E7CC
:1019700070E085EF90E0F0DA53EAE52EF12C25E7F0
:1019800030E04FE251E065E770E087EF90E0E4DAA5
:1019900066E4E62E65E0F62E02E020EE37E040E059
:1019A00050E068EC70E08DE290E0C3D81F910F9199
:1019B000FF90EF90DF90CF900895CF93DF9300D00A
:1019C00000D0CDB7DEB7809163001C821B821A82E3
:1019D0001982BE016F5F7F4FCE0103960E94CA3FFE
:1019E0008B819C81853C994068F089819A81843AF9
:1019F000964040F489819A818D32914018F082E0BE
:101A0000809338068B819C81803D974090F48B8138
:101A10009C818139914068F089819A81843A96400D
:101A200040F489819A818D32914018F083E080934F
:101A300038068B819C818032934068F489819A8139
:101A400084379E4040F489819A81813D974018F007
:101A500081E0809338068B819C81843C994060F4BE
:101A60008B819C81893E934038F089819A81813DA8
:101A7000974010F010923806809138060F900F9022
:101A80000F900F90DF91CF910895CF92DF92EF9258
:101A9000FF920F931F93A89500EE17E021E430E02A
:101AA00048EC50E06AEA70E085E090E00E94A4040F
:101AB0000FEF1FEF21E430E048EC50E063E270E00C
:101AC00085E090E09DD920E530E040E550E065E01C
:101AD00070E08BEE90E094D9F0EECF2EF7E0DF2EA1
:101AE000A4E1EA2EF12C03E111E026E430E041E329
:101AF00051E066E470E085EF90E02EDAB7E1EB2E7E
:101B0000F12C24E430E04FE251E064E470E087EF30
:101B100090E022DA0FEF1FEF20E530E040E550E0E3
:101B200064E670E08BEE90E06BD915EAE12EF12CC3
:101B300003E111E023E730E041E351E063E770E0C7
:101B400085EF90E009DA83EAE82EF12C25E730E012
:101B50004FE251E065E770E087EF90E0FDD99EEC41
:101B6000E92E95E0F92E02E020EE37E040E050E06B
:101B700068EC70E08CE390E00E9499058091120679
:101B800090911306892B09F048C0E0916F068E2FC3
:101B900090E08830910508F040C0FC01E25BFF4F07
:101BA0000C946741E3E9EE2EE4E0FE2E04C07EE8EB
:101BB000E72E74E0F72E02E02FE130E04FEF5FEF09
:101BC00065E070E086E490E026C064E8E62E64E01C
:101BD000F62E18C05AE7E52E54E0F52E13C040E764
:101BE000E42E44E0F42E0EC036E6E32E34E0F32E6D
:101BF00009C02CE5E22E24E0F22E04C092E5E92E85
:101C000094E0F92E02E02FE130E04FEF5FEF65E066
:101C100070E08EE190E00E9499058091120690910B
:101C20001306019701F580911B06813069F038F0A9
:101C30008230C9F410E7E12E14E0F12E09C084E8E7
:101C4000E82E84E0F82E04C00AE7E02E04E0F02E2F
:101C500002E02FE130E04FEF5FEF65E070E08EE1F2
:101C600090E00E94990580911206909113060297C8
:101C700001F580912206813069F038F08230C9F494
:101C8000F0E7EF2EF4E0FF2E09C0B4E8EB2EB4E04D
:101C9000FB2E04C0AAE7EA2EA4E0FA2E02E02FE110
:101CA00030E04FEF5FEF65E070E08EE190E00E9482
:101CB00099058091120690911306049701F5809181
:101CC0007A06813069F038F08230C9F460E7E62E98
:101CD00064E0F62E09C0E4E8EE2EE4E0FE2E04C037
:101CE0007AE7E72E74E0F72E02E02FE130E04FEFC5
:101CF0005FEF65E070E08EE190E00E9499058091D1
:101D0000120690911306059701F580916E068130B9
:101D100069F038F08230C9F430E7E32E34E0F32E76
:101D200009C054E8E52E54E0F52E04C04AE7E42E3D
:101D300044E0F42E02E02FE130E04FEF5FEF65E08A
:101D400070E08EE190E00E949905809112069091DA
:101D50001306069701F580916B06813069F038F023
:101D60008230C9F480E7E82E84E0F82E09C024E828
:101D7000E22E24E0F22E04C09AE7E92E94E0F92E38
:101D800002E02FE130E04FEF5FEF65E070E08EE1C1
:101D900090E00E9499051F910F91FF90EF90DF90C6
:101DA000CF900895EF92FF920F931F9380910906B1
:101DB00090910A060A97A8F48091E00581110CC061
:101DC0000FE110E02CE330E044E650E06BE470E01B
:101DD0008EE690E00E94A40481E08093E0051092DA
:101DE00014068091090690910A060A978A35910592
:101DF000A8F48091140681110CC00FE110E02CE3CF
:101E000030E044E650E06BE470E08EE690E00E9443
:101E1000A40481E0809314061092E00580910906E5
:101E200090910A0684369105A0F0809114068130C5
:101E300061F40FE110E02CE330E044E650E06BE4A5
:101E400070E08EE690E00E94A404109214061092B6
:101E5000E0058091100690911106019779F4E090C9
:101E60000906F0900A0603E02FE130E04FEF5FEF44
:101E700064E670E082E890E00E94DF058091100641
:101E800090911106892B79F4E0900906F0900A06EA
:101E900003E02FE130E040E058EF64E670E082E8D4
:101EA00090E00E94DF051F910F91FF90EF90089541
:101EB000EF92FF920F931F9380913C0690913D0605
:101EC0000A97A8F480910806811111C00FE110E073
:101ED00027E330E048E550E06BE970E088E090E00F
:101EE0000E94A40481E08093080610926C06809101
:101EF0003C0690913D0684369105D8F48091090600
:101F000090910A060A97A8F080916C06811111C081
:101F10000FE110E027E330E048E550E06BE970E0C6
:101F200088E090E00E94A40481E080936C06109207
:101F3000080680913C0690913D0684369105A0F0FC
:101F400080916C06813061F40FE110E027E330E00E
:101F500048E550E06BE970E088E090E00E94A4045E
:101F600010926C0610920806E0903C06F0903D0638
:101F700003E02FE130E04FEF5FEF64EB70E08FE0C4
:101F800090E00E94DF051F910F91FF90EF90089560
:101F9000EF92FF920F931F938091290690912A064A
:101FA0000A97A8F480910F0681110CC00FE110E090
:101FB00024E230E04AE550E064E670E088E090E03A
:101FC0000E94A40481E080930F061092260680915F
:101FD000290690912A060A978A359105A8F48091DE
:101FE000260681110CC00FE110E024E230E04AE542
:101FF00050E064E670E088E090E00E94A40481E094
:102000008093260610920F068091290690912A0649
:1020100084369105A1F480912606813061F40FE1A8
:1020200010E024E230E04AE550E064E670E088E049
:1020300090E00E94A40410920F0610922606809150
:10204000290690912A068436910530F084E690E0C6
:1020500090932A0680932906E0902906F0902A069C
:1020600003E02FE130E04FEF5FEF6EE670E084E1D8
:1020700090E00E94DF0580917B0690917C060A9794
:10208000A8F480917506811111C00FE110E024E2DF
:1020900030E04AE550E064E670E08FED90E00E94A9
:1020A000A40481E08093750610923E0680917B0621
:1020B00090917C060A978A359105A8F480913E0696
:1020C000811111C00FE110E024E230E04AE550E058
:1020D00064E670E08FED90E00E94A40481E08093BC
:1020E0003E061092750680917B0690917C068436A0
:1020F000910529F41092750610923E0603C08436AD
:10210000910530F084E690E090937C0680937B0606
:10211000E0907B06F0907C0603E02FE130E04FEF8B
:102120005FEF6EE670E089EE90E00E94DF051F91A0
:102130000F91FF90EF900895CF93DF9300D000D0E0
:10214000CDB7DEB7809163001C821B821A82198290
:10215000BE016F5F7F4FCE0103960E94CA3F8B8105
:102160009C8188379540A0F4A89589819A81843C08
:10217000994070F4A89589819A818D3D954040F0F1
:10218000A89581E090E09093110680931006A895A1
:102190000F900F900F900F90DF91CF910895CF93F4
:1021A000DF9300D000D0CDB7DEB7A8958091630053
:1021B0001C821B821A821982BE016F5F7F4FCE0183
:1021C00003960E94CA3F8B819C818837954070F4AA
:1021D00089819A81843C994048F489819A818D3D16
:1021E000954020F010921106109210060F900F905B
:1021F0000F900F90DF91CF9108957F928F929F92D1
:10220000AF92BF92CF92DF92EF92FF920F931F9304
:10221000CF93DF93EC016B015A014901702EA89511
:102220008091E3059091E4050A97A8F480917006E7
:10223000811111C00FE110E02EE130E044E650E0E2
:1022400065507109CE0144970E94A40481E08093F7
:102250007006109231068091E3059091E4050A978B
:102260008A359105C0F480913106811114C00FE1C7
:1022700010E02EE130E044E650E0B601655071090F
:10228000CE0144970E94A40481E08093310610920D
:10229000700610920B068091E3059091E405843658
:1022A0009105C0F080910B06811114C00FE110E080
:1022B0002EE130E044E650E0B60165507109CE01F0
:1022C00044970E94A40481E080930B06109231068B
:1022D00010927006E090E305F090E405072D94015C
:1022E000A501B601CE010E94DF05A895DF91CF912F
:1022F0001F910F91FF90EF90DF90CF90BF90AF9024
:102300009F908F907F900895A89580912E068130A0
:1023100071F4A49A80E185BBA8952FEF82E597E040
:10232000215080409040E1F700C0000015BAA89508
:102330000895A89580912E06813021F5A49A80E118
:1023400085BB2FEF32E597E0215030409040E1F718
:1023500000C00000A89515BA2FEF32E597E0215094
:1023600030409040E1F700C00000A89585BB2FEFFA
:1023700032E587E0215030408040E1F700C00000A6
:10238000A89515BA0895A89580912E06813009F078
:1023900048C0A49A80E185BBA8952FEF32E597E06D
:1023A000215030409040E1F700C00000A89515BAD8
:1023B000A8952FEF32E597E0215030409040E1F7AB
:1023C00000C00000A89585BBA8952FEF32E597E0E7
:1023D000215030409040E1F700C00000A89515BAA8
:1023E000A8952FEF32E597E0215030409040E1F77B
:1023F00000C00000A89585BB2FEF32E587E0215093
:1024000030408040E1F700C00000A89515BA9FEF6A
:1024100022E537E0915020403040E1F700C0000055
:10242000A8950895A89510922B0610921F06109259
:10243000DE051092410610921C0610920E061092B4
:102440002D061092250610923B061092DF0583EBB5
:1024500092E00E94824480932E06A89584EB92E03D
:102460000E948A449093210680932006A89580912B
:10247000120690911306892B51F5A895E0916F06ED
:102480008E2F90E08830910510F5FC01EA5AFF4F3D
:102490004EE150E00C94674164E972E014C066E7D5
:1024A00072E011C068E572E00EC06AE372E00BC032
:1024B0006CE172E008C06EEF71E005C060EE71E0A3
:1024C00002C062EC71E089EE95E00E947244A8952A
:1024D00080911206909113060197D1F4A8958091EE
:1024E0001B06813069F038F0823091F44EE150E003
:1024F00068E671E009C04EE150E064EA71E004C0B2
:102500004EE150E066E871E089EE95E00E94724489
:10251000A89580911206909113060297D1F4A89580
:1025200080912206813069F038F0823091F44EE1DA
:1025300050E06EE071E009C04EE150E06AE471E005
:1025400004C04EE150E06CE271E089EE95E00E943B
:102550007244A89580911206909113060497C9F4CD
:1025600080917A06813069F038F0823091F44EE142
:1025700050E064EB70E009C04EE150E060EF70E0C5
:1025800004C04EE150E062ED70E089EE95E00E94FB
:102590007244A89580911206909113060597C9F48C
:1025A00080916E06813069F038F0823091F44EE10E
:1025B00050E06AE570E009C04EE150E066E970E085
:1025C00004C04EE150E068E770E089EE95E00E94BB
:1025D0007244A89580911206909113060697C9F44B
:1025E00080916B06813069F038F0823091F44EE1D1
:1025F00050E060E070E009C04EE150E06CE370E054
:1026000004C04EE150E06EE170E089EE95E00E947A
:102610007244A89587EC90E00197F1F700C00000A4
:102620008091E9059091EA059093DD058093DC05A2
:102630008091EB059091EC059093300680932F06E6
:102640008091ED059091EE05909378068093770642
:102650008091EF059091F00590931A0680931906EA
:102660008091F105809344068091F3059091F405E3
:1026700090931806809317068091F505809328069D
:102680008091F705809327068091F9058093D805FE
:102690008091FB059091FC059093680680936706F6
:1026A0008091FD059091FE0590934306809342062C
:1026B0008091120690911306079741F48091FF05CF
:1026C0009091000690931306809312068091010664
:1026D00090910206909366068093650680910306AA
:1026E000909104069093E8058093E7058091050694
:1026F0009091060690930D0680930C06A895089578
:1027000010927C0610927B06BC9A80917B06880F03
:1027100081BF10922A0610922906139A80912906E9
:10272000880F809386002FDE8DE490E090937206F0
:102730008093710681E090E09093110680931006DB
:102740000895CF934091E3055091E4052091190637
:1027500030911A06429FC001439F900D529F900DE9
:1027600011246AE070E00E94534170934006609328
:102770003F068091290690912A068536910530F012
:1027800084E690E090932A0680932906809127069C
:1027900090E02091290630912A068217930720F4B1
:1027A00090932A068093290620912B06211114C0AC
:1027B00020913C0630913D062233310538F424E661
:1027C00030E030932A062093290606C022333105D3
:1027D00019F021E020932B0620912B0640912F0623
:1027E000509130062130E1F52091290630912A06DA
:1027F0002436310530F024E630E030932A06209369
:1028000029066417750760F5E0913C06F0913D06D6
:102810002091290630912A06E617F707C0F42F5FAA
:102820003F4F8217930728F030932A0620932906FA
:1028300004C090932A06809329062091290630919E
:102840002A062536310560F024E630E005C0211562
:10285000310531F02150310930932A0620932906A1
:102860004617570708F04AC020913C0630913D06B4
:1028700024173507D0F46091290670912A066F5FFE
:102880007F4F6536710510F064E670E070932A069C
:10289000609329066091290670912A06861797078A
:1028A00020F490932A06809329064217530730F5A7
:1028B0008091290690912A06009729F0019790931C
:1028C0002A0680932906241B350B2B303105B0F0E6
:1028D0008091290690912A060A9720F410922A06E0
:1028E000109229068091290690912A068A30910536
:1028F00028F00A9790932A0680932906C0914406EF
:10290000C130D1F480911F06811116C020910906B3
:1029100030910A06809117069091180628173907FA
:1029200059F480913C0690913D0690933006809337
:102930002F06EADCC0931F06C091D805C13009F507
:102940008091DE0581111DC08091090690910A06D3
:102950002091670630916806821B930B059788F4D7
:1029600020912F06309130068091420690914306C7
:10297000820F931F9093300680932F06C5DCC0937F
:10298000DE05CF9108958091410681111CC0809190
:10299000090690910A062091170630911806821BAD
:1029A000930B029780F482E390E090937C068093EF
:1029B0007B0681E08093410680930E068091440659
:1029C000811101C0A1DC2091170630911806609199
:1029D0007306709174064091770650917806649F53
:1029E000C001659F900D749F900D11246AE070E006
:1029F0000E945341620F731F7093DB056093DA05E9
:102A0000E0917B06F0917C064091DC055091DD055C
:102A10004617570720F45093DB054093DA05809161
:102A2000280690E08E179F0720F490937C068093F1
:102A30007B068091090690910A062817390720F035
:102A400048175907A0F176C020913B062111F8CF15
:102A500084179507A8F76091DA057091DB0520913E
:102A60007B0630917C068617970788F42F5F3F4FCF
:102A70002536310528F430937C0620937B06E0CF81
:102A800024E630E030937C0620937B06A6C0211517
:102A9000310531F02150310930937C0620937B06BB
:102AA00020917B0630917C06232B51F296C0209119
:102AB0007B0630917C062115310531F0215031091A
:102AC00030937C0620937B06841B950B0697B0F011
:102AD00080917B0690917C060A9720F410927C06E8
:102AE00010927B0680917B0690917C068A3091053E
:102AF00028F00A9790937C0680937B068091DF05EF
:102B0000811106C016DC81E0809325068093DF05E5
:102B10002091E5053091E6058091200690912106EF
:102B20008217930738F4ECDD81E090E09093110672
:102B30008093100680911C06811158C04091650653
:102B40005091660680911706909118068417950794
:102B500008F04CC0E0910906F0910A064E175F0795
:102B600029F481E080933B0680932D0680913B06FB
:102B70008130E1F56091E1057091E2052091E70572
:102B80003091E80562177307A8F480917B06909155
:102B90007C06E417F50738F401968536910530F088
:102BA00084E690E003C0009729F0019790937C069B
:102BB00080937B0626173707C8F410923B06809156
:102BC000730690917406821B930B90937406809306
:102BD000730681E080931C0608954817590708F092
:102BE000A9CF20917B0630917C0668CF0895809113
:102BF000410681111BC02091090630910A0680917F
:102C00001706909118068217930780F482E390E0EC
:102C100090937C0680937B0681E0809341068093AD
:102C20000E0680914406811101C06EDBE09117060B
:102C3000F091180640917306509174062091770622
:102C400030917806429FC001439F900D529F900D96
:102C500011246AE070E00E9453416E0F7F1F709351
:102C6000DB056093DA0520917B0630917C0640916C
:102C7000DC055091DD054617570720F45093DB051E
:102C80004093DA058091280690E08217930720F49C
:102C900090937C0680937B062091090630910A066A
:102CA000E217F30700F580913B0681111CC0241741
:102CB0003507C8F46091DA057091DB0580917B06D9
:102CC00090917C062617370738F4019685369105D2
:102CD00030F084E690E003C0009729F001979093CC
:102CE0007C0680937B0642175307E0F580917B06B4
:102CF00090917C06019790937C0680937B06241B21
:102D0000350B2630310590F00A9720F410927C069E
:102D100010927B0680917B0690917C068A3091050B
:102D200028F00A9790937C0680937B068091DF05BC
:102D3000811106C0FEDA81E0809325068093DF05CD
:102D40002091E5053091E6058091200690912106BD
:102D50008217930738F4D4DC81E090E09093110659
:102D60008093100680911C0681114EC0409165062B
:102D70005091660680911706909118068417950762
:102D800008F042C0E0910906F0910A064E175F076D
:102D900029F481E080933B0680932D0680913B06C9
:102DA000813091F56091E1057091E2052091E70590
:102DB0003091E80562177307A8F480917B06909123
:102DC0007C06E417F50738F401968536910530F056
:102DD00084E690E003C0009729F0019790937C0669
:102DE00080937B062617370778F410923B06809174
:102DF000730690917406821B930B909374068093D4
:102E0000730681E080931C060895CF93C091440619
:102E1000C130D1F480911F06811116C0209109069E
:102E200030910A06809117069091180628173907E5
:102E300059F480913C0690913D0690933006809322
:102E40002F0662DAC0931F064091E3055091E40516
:102E50002091190630911A06429FC001439F900DA0
:102E6000529F900D11246AE070E00E9453417093CC
:102E7000400660933F068091290690912A06853688
:102E8000910530F084E690E090932A06809329061D
:102E90008091270690E02091290630912A0682171A
:102EA000930720F490932A068093290620912B06FD
:102EB000211114C020913C0630913D062639310580
:102EC00038F424E630E030932A062093290606C021
:102ED0002639310519F021E020932B0620912B068D
:102EE00040912F0650913006213079F5641775070F
:102EF00060F5E0913C06F0913D0620912906309165
:102F00002A06E617F707C0F42F5F3F4F8217930793
:102F100028F030932A062093290604C090932A06AD
:102F2000809329062091290630912A0625363105FD
:102F300060F024E630E005C02115310531F0215064
:102F4000310930932A06209329064617570708F0BF
:102F500088C020914406211133C020913C06309155
:102F60003D0624173507D0F46091290670912A0692
:102F70006F5F7F4F6536710510F064E670E0709307
:102F80002A06609329066091290670912A06861701
:102F9000970720F490932A06809329064217530737
:102FA00008F05FC08091290690912A06009729F0C9
:102FB000019790932A0680932906241B350B38C06D
:102FC000213009F04EC02091090630910A06609127
:102FD00017067091180626173707D0F44091290676
:102FE00050912A064F5F5F4F4536510510F044E679
:102FF00050E050932A0640932906409129065091AB
:103000002A068417950720F490932A0680932906B0
:103010006217730730F58091290690912A06009770
:1030200029F0019790932A0680932906261B370BD7
:103030002B303105B0F08091290690912A060A972D
:1030400020F410922A061092290680912906909168
:103050002A068A30910528F00A9790932A068093D1
:103060002906CF9108954091E3055091E405209100
:10307000190630911A06429FC001439F900D529F3E
:10308000900D11246AE070E00E9453417093400655
:1030900060933F068091290690912A068536910516
:1030A00030F084E690E090932A0680932906809180
:1030B000270690E02091290630912A06821793076F
:1030C00020F490932A068093290620912B064091A4
:1030D0003C0650913D06211110C04639510538F487
:1030E00024E630E030932A062093290606C04639AC
:1030F000510519F021E020932B0620912B06E09139
:103100002F06F0913006213059F56E177F0740F5F4
:103110002091290630912A0646175707C0F42F5FE1
:103120003F4F8217930728F030932A0620932906F1
:1031300004C090932A068093290620912906309195
:103140002A062536310560F024E630E005C0211559
:10315000310531F02150310930932A062093290698
:10316000E617F70708F046C04E175F07D0F4209126
:10317000290630912A062F5F3F4F2536310510F082
:1031800024E630E030932A06209329062091290670
:1031900030912A068217930720F490932A06809391
:1031A0002906E417F50730F58091290690912A0643
:1031B000009729F0019790932A0680932906CA0167
:1031C0008E1B9F0B0B97B0F08091290690912A06D9
:1031D0000A9720F410922A06109229068091290657
:1031E00090912A068A30910528F00A9790932A0632
:1031F000809329068091280690E020917B063091EB
:103200007C068217930720F490937C0680937B06BC
:10321000E417F50770F480917B0690917C06019687
:103220008536910510F084E690E090937C068093BB
:103230007B0608954091E3055091E405209119061D
:1032400030911A06429FC001439F900D529F900DEE
:1032500011246AE070E00E9453417093400660932D
:103260003F068091290690912A068536910530F017
:1032700084E690E090932A068093290680912706A1
:1032800090E02091290630912A068217930720F4B6
:1032900090932A068093290620912B06211114C0B1
:1032A00020913C0630913D062639310538F424E65C
:1032B00030E030932A062093290606C026393105CE
:1032C00019F021E020932B0620912B0640912F0628
:1032D00050913006213079F56417750760F5E0915B
:1032E0003C06F0913D062091290630912A06E6170A
:1032F000F707C0F42F5F3F4F8217930728F03093F2
:103300002A062093290604C090932A068093290652
:103310002091290630912A062536310560F024E6F1
:1033200030E005C02115310531F0215031093093CD
:103330002A06209329064617570708F04AC020910D
:103340003C0630913D0624173507D0F460912906DC
:1033500070912A066F5F7F4F6536710510F064E645
:1033600070E070932A066093290660912906709197
:103370002A068617970720F490932A068093290639
:103380004217530730F58091290690912A0600973D
:1033900029F0019790932A0680932906241B350B68
:1033A0002B303105B0F08091290690912A060A97BA
:1033B00020F410922A0610922906809129069091F5
:1033C0002A068A30910528F00A9790932A0680935E
:1033D00029060895BC9A80917B06880F81BF139AB5
:1033E00080912906880F8093860080911206909123
:1033F0001306892B11F4A5D9C6DA80911206909193
:103400001306019729F410922A0610922906EFDB81
:103410008091120690911306029729F410927C066F
:1034200010927B06F2DC80911206909113060497AD
:1034300009F419DE8091120690911306059709F49C
:1034400012DE8091120690911306069709F4F2CECF
:10345000089563EC70E084E992E00E94A54462EC78
:1034600071E086E992E00E94A54466E170E088E997
:1034700092E00E94A54466E170E08AE992E00E9431
:10348000A54461E070E08CE992E00E94A544A89513
:103490006EE670E08EE992E00E94A54464E670E07A
:1034A00080EA92E00E94A54464E670E082EA92E03D
:1034B0000E94A54460E070E084EA92E00E94A54486
:1034C000A89560E070E086EA92E00E94A54460E082
:1034D00070E088EA92E00E94A54460E070E08AEA29
:1034E00092E00E94A54460E070E08CEA92E00E94C5
:1034F000A54460E070E08EEA92E00E94A54460E09E
:1035000070E080EB92E00E94A544A89566EE70E022
:1035100086E792E00E94A54462EC71E088E792E0C1
:103520000E94A54466E170E08AE792E00E94A5440B
:1035300066E170E08CE792E00E94A54461E070E0F3
:103540008EE792E00E94A544A89563E770E080E8CA
:1035500092E00E94A54464E670E082E892E00E9456
:10356000A54464E670E084E892E00E94A54460E02F
:1035700070E086E892E00E94A54460E070E088E890
:1035800092E00E94A54460E070E08AE892E00E9428
:10359000A544A89560E070E08CE892E00E94A54404
:1035A00060E070E08EE892E00E94A54460E070E088
:1035B00080E992E00E94A54460E070E082E992E038
:1035C0000E94A544A89566EE70E088E592E00E940E
:1035D000A54462EC71E08AE592E00E94A54466E1B0
:1035E00070E08CE592E00E94A54466E170E08EE513
:1035F00092E00E94A54461E070E080E692E00E94C3
:10360000A544A89563E770E082E692E00E94A54495
:1036100064E670E084E692E00E94A54464E670E00F
:1036200086E692E00E94A54460E070E088E692E0C1
:103630000E94A54460E070E08AE692E00E94A54402
:1036400060E070E08CE692E00E94A544A89560E0FE
:1036500070E08EE692E00E94A54460E070E080E7B2
:1036600092E00E94A54460E070E082E792E00E9450
:10367000A54460E070E084E792E00E94A544A8952C
:1036800066E970E08AE392E00E94A54468EC70E08D
:103690008CE392E00E94A54466E170E08EE392E044
:1036A0000E94A54466E170E080E492E00E94A54497
:1036B00061E070E082E492E00E94A544A89563E78F
:1036C00070E084E492E00E94A54464E670E086E441
:1036D00092E00E94A54464E670E088E492E00E94D3
:1036E000A54460E070E08AE492E00E94A54460E0B6
:1036F00070E08CE492E00E94A54460E070E08EE40B
:1037000092E00E94A544A89560E070E080E592E018
:103710000E94A54460E070E082E592E00E94A5442A
:1037200060E070E084E592E00E94A54460E070E013
:1037300086E592E00E94A544A8956EEB70E08CE1CE
:1037400092E00E94A54468EC70E08EE192E00E9455
:10375000A54466E170E080E292E00E94A54466E143
:1037600070E082E292E00E94A54461E070E084E2B1
:1037700092E00E94A544A89564E670E086E292E09B
:103780000E94A54464E670E088E292E00E94A544AD
:1037900064E670E08AE292E00E94A54460E070E096
:1037A0008CE292E00E94A54460E070E08EE292E03C
:1037B0000E94A54460E070E080E392E00E94A5448E
:1037C000A89560E070E082E392E00E94A54460E08A
:1037D00070E084E392E00E94A54460E070E086E33C
:1037E00092E00E94A54460E070E088E392E00E94CD
:1037F000A544A89566EE70E08EEF91E00E94A54486
:1038000062EC71E080E092E00E94A54466E170E025
:1038100082E092E00E94A54466E170E084E092E0DC
:103820000E94A54461E070E086E092E00E94A54419
:10383000A89563E770E088E092E00E94A54464E602
:1038400070E08AE092E00E94A54464E670E08CE0BB
:1038500092E00E94A54460E070E08EE092E00E9459
:10386000A54460E070E080E192E00E94A54460E041
:1038700070E082E192E00E94A544A89560E070E0CB
:1038800084E192E00E94A54460E070E086E192E06D
:103890000E94A54460E070E088E192E00E94A544A7
:1038A00060E070E08AE192E00E94A544A89566EE8F
:1038B00070E080EE91E00E94A54462EC71E082EE3F
:1038C00091E00E94A54466E170E084EE91E00E94E0
:1038D000A54466E170E086EE91E00E94A54461E0B7
:1038E00070E088EE91E00E94A544A89563E770E03F
:1038F0008AEE91E00E94A54464E670E08CEE91E0CF
:103900000E94A54464E670E08EEE91E00E94A5441A
:1039100060E070E080EF91E00E94A54460E070E01C
:1039200082EF91E00E94A54460E070E084EF91E0B6
:103930000E94A544A89560E070E086EF91E00E94A7
:10394000A54460E070E088EF91E00E94A54460E04B
:1039500070E08AEF91E00E94A54460E070E08CEF97
:1039600091E00E94A544A89563EC70E084EA91E0A0
:103970000E94A54466E170E088EA91E00E94A544B7
:1039800061E070E08CEA91E00E94A5446FE070E095
:103990008EEA91E00E94A544A89564E670E080EB71
:1039A00091E00E94A54461E070E08AEB91E00E9402
:1039B000A54463EC70E08CEB91E00E94A5446AE0C2
:1039C00070E08EEB91E00E94A544A89562EC71E056
:1039D0008CE491E00E94A54466E170E080E591E00E
:1039E0000E94A54461E070E082E591E00E94A54458
:1039F0006EE670E084E591E00E94A544A89564E637
:103A000070E088E591E00E94A54462E070E080E605
:103A100091E00E94A54462EC71E082EF90E00E9488
:103A2000A54466E170E084EF90E00E94A54462E165
:103A300070E086EF90E00E94A544A89564E670E0EF
:103A40008CEF90E00E94A54464E670E08EEF90E079
:103A50000E94A54464E070E086E091E00E94A544E5
:103A60006CE271E08CE091E00E94A544A89562ECC4
:103A700071E088E990E00E94A54466E170E08AE97F
:103A800090E00E94A54466E170E08CE990E00E941D
:103A9000A54461E070E08EE990E00E94A544A895FD
:103AA0006EE670E080EA90E00E94A54464E670E073
:103AB00082EA90E00E94A54464E670E084EA90E027
:103AC0000E94A54465E070E08CEA90E00E94A54465
:103AD000A89562EC71E08EE390E00E94A54466E157
:103AE00070E082E490E00E94A54461E070E084E42C
:103AF00090E00E94A5446EE670E086E490E00E94AB
:103B0000A544A89564E670E08AE490E00E94A5448C
:103B100066E070E082E590E00E94A54463EC70E00E
:103B200084E992E00E94A544A89508956FE070E0B2
:103B300088EB92E00E94A5446FE070E086EB92E093
:103B40000E94A5446FE070E084EB92E00E94A544DF
:103B500061E083EB92E00E94984461E082EB92E0A6
:103B60000C9498448FB9779BFECF8FB10895CF9373
:103B7000A39AAB9AAB9880E0F5DFC82F80E0F2DF24
:103B8000AB9A6C2F70E0762F6627682B687F7F7763
:103B900023E0769567952A95E1F780E090E00E9412
:103BA000624020E030E040E85EE30E94C8400E94AE
:103BB000364070930A0660930906CB01CF910895B1
:103BC000CF93A79AAF9AAF9880E0CCDFC82F80E060
:103BD000C9DFAF9A6C2F70E0762F6627682B687F5D
:103BE0007F7723E0769567952A95E1F780E090E06E
:103BF0000E94624020E030E040E85EE30E94C8405E
:103C00000E94364070933D0660933C06CB01CF91F5
:103C1000089580E091E090938106809380068091E2
:103C20000A068F93809109068F938EE091E09F930F
:103C30008F930E94A2418DE08A95F1F70000809158
:103C4000E4058F938091E3058F9388E191E09F9342
:103C50008F930E94A2419DE09A95F1F70000809118
:103C60002A068F93809129068F9382E291E09F9399
:103C70008F930E94A2418DE08A95F1F70000809118
:103C80007C068F9380917B068F938DE291E09F93CA
:103C90008F930E94A2419DE09A95F1F7000087E37F
:103CA00091E09F938F930E94A2418DE08A95F1F756
:103CB000000080913D068F9380913C068F938FE3A7
:103CC00091E09F938F930E94A2418DB79EB7469635
:103CD0000FB6F8949EBF0FBE8DBF809110069091D5
:103CE0001106892B41F488E491E09F938F930E9401
:103CF000A2410F900F9080911006909111060197AC
:103D000041F48FE491E09F938F930E94A2410F9022
:103D10000F909DE09A95F1F70000E0911206F09166
:103D20001306E830F10508F08FC0E25AFF4F0C94FB
:103D3000674186E591E09F938F930E94A2410F9087
:103D40000F90E0916F068E2F90E08830910508F07B
:103D50007BC0FC01EA59FF4F0C94674185E691E076
:103D60006DC085E791E06AC08DEA91E067C08CEB99
:103D700091E064C08BEC91E061C08AED91E09F938B
:103D80008F930E94A2410F900F9080911B0681306B
:103D900009F44CC008F447C0823009F44AC00895C1
:103DA0008AEE91E09F938F930E94A2410F900F9013
:103DB000809122068130D1F1B0F18230D1F10895A5
:103DC0008BEF91E03BC089E092E09F938F930E943C
:103DD000A2410F900F9080917A06813039F118F14D
:103DE000823039F108958AE192E09F938F930E9487
:103DF000A2410F900F9080916E068130B9F098F03B
:103E00008230B9F008958DE292E09F938F930E94E3
:103E1000A2410F900F9080916B06813039F018F01D
:103E2000823039F0089580E891E008C08FE891E091
:103E300005C08EE991E002C08FE392E09F938F93DB
:103E40000E94A2410F900F900895CF92DF92EF92BF
:103E5000FF920F931F93CF93DF9300D000D0CDB785
:103E6000DEB78091100690911106019709F00EC1FE
:103E70008091230690912406892BC9F40FE110E06C
:103E800024E230E04AE550E064E670E088E090E04B
:103E90000E94A40424E230E04AE550E064E670E0C9
:103EA0008FED90E00E94A404A8950E94EB07CC241B
:103EB000C394D12C8091100690911106019709F0BE
:103EC000E5C0A895A6DE80917106909172068A35AC
:103ED000910549F42FEF8DE399E421508040904003
:103EE000E1F700C00000A89503E02FE130E04FEFBC
:103EF0005FEF69E170E085E890E00E94FD1080913D
:103F00006300A8951C821B821A821982BE016F5F12
:103F10007F4FCE0103960E94CA3F8B819C81853CD6
:103F2000994088F089819A81883D9E4060F489811A
:103F30009A81853C994038F0D0922406C09223069D
:103F400010923306F1D38B819C81853C994008F413
:103F50003FC089819A818C3D9540D0F589819A81B5
:103F6000853F9140A8F1D0922406C092230610927A
:103F700045068091120690911306892B11F40E9438
:103F800034328091120690911306019711F40E9429
:103F9000D03A8091120690911306029711F40E9474
:103FA000D73B8091120690911306049711F40E945A
:103FB000DC3C8091120690911306059709F43CD5DC
:103FC0008091120690911306069711F40E942C31ED
:103FD000CEDD0E94D20EA8958FEF91EE24E08150A5
:103FE00090402040E1F700C00000EADDA8950E9463
:103FF000580FE0902906F0902A0603E02FE130E008
:104000004FEF5FEF6EE670E08CE190E00E94DF051D
:10401000E0907B06F0907C062FE130E04FEF5FEF01
:104020006EE670E080EF90E00E94DF050E94CF1006
:104030008091100690911106892B09F03BCF0E94C8
:104040008411A8950E941212A8950E94EB070FE117
:1040500010E024E230E04AE550E064E670E088E0F9
:1040600090E00E94A40424E230E04AE550E064E6D7
:1040700070E08FED90E00E94A4041092E40510928D
:10408000E305109224061092230614CF0F900F9090
:104090000F900F90DF91CF911F910F91FF90EF90B4
:1040A000DF90CF900895EF92FF920F931F93CF93DD
:1040B00080913206813009F04BC18FE190E00E947F
:1040C00019060E94C10B85E080933806C5E08091F7
:1040D0003206813009F03CC10E94DD0C8091380627
:1040E0008230D9F4809164068F5F809364060FE17B
:1040F00010E02CE330E046EE50E069E670E081E04D
:1041000090E00E94A40422E330E043EC50E068E237
:1041100070E088E090E00E94A4048091380683302B
:10412000D9F4809164068150809364060FE110E019
:104130002CE330E046EE50E069E670E081E090E08C
:104140000E94A40422E330E043EC50E068E270E017
:1041500088E090E00E94A40480916406853010F00D
:104160001092640680916406823081F1B8F488234D
:10417000D9F0813009F0C1C075E8E72E75E0F72E5F
:1041800001E02FE130E04FEF5FEF6CE370E088E09B
:1041900090E00E94990586EB92E029C08330B1F14E
:1041A000843009F471C0A9C0EEE9EE2EE5E0FE2EE0
:1041B00001E02FE130E04FEF5FEF6CE370E08FE064
:1041C00090E00E94990588EB92E011C069E7E62E25
:1041D00065E0F62E01E02FE130E04FEF5FEF6CE39A
:1041E00070E082E390E00E94990584EB92E00E94E7
:1041F0008A447C0103E02FE130E04FEF5FEF62E89B
:1042000070E080E590E00E94DF0577C041E6E42E93
:1042100045E0F42E01E02FE130E04FEF5FEF6CE37B
:1042200070E088E290E00E9499055FE6E52E55E097
:10423000F52E02E02FE130E04FEF5FEF62E870E033
:1042400088E290E00E94990580913806811119C09A
:1042500000D96CDC3BE2E32E35E0F32E2FE130E0B9
:104260004FEF5FEF62E870E088E290E00E9499050E
:104270002FEF89E698E1215080409040E1F700C09F
:104280000000C093380639C020E5E22E25E0F22E6A
:1042900001E02FE130E04FEF5FEF6CE370E08EE183
:1042A00090E00E94990583EB92E00E948244813065
:1042B00079F492E4E92E95E0F92E03E02FE130E065
:1042C0004FEF5FEF62E870E080E590E00E949905B3
:1042D00083EB92E00E94824481110FC08DE3E82EAF
:1042E00085E0F82E03E02FE130E04FEF5FEF62E86A
:1042F00070E080E590E00E94990580913806813059
:1043000089F41092320610922406109223068FE14F
:1043100090E00E94190681E090E09093110680934E
:10432000100693DD80913806811106C081E08093EC
:1043300032061092760612D0C09338062FE785EB2E
:1043400091E0215080409040E1F700C00000BFCED6
:10435000CF911F910F91FF90EF900895BF92CF9250
:10436000DF92EF92FF920F931F93CF93DF93809191
:1043700076068111CFC185E080933806C9E1D0E08F
:1043800025E0C22ED12C35E0B32E80917606811126
:10439000C1C180916406813009F46FC038F0823069
:1043A00009F4DDC0843009F441C1A4C188EB92E076
:1043B0000E948A447C0103E02FE130E040E058EFA6
:1043C00062E870E080E590E00E94DF0588EB92E013
:1043D0000E948A4490933706809336060E94DD0C33
:1043E000809138068230A9F4809136069091370684
:1043F000019690933706809336060FE110E02CE388
:1044000030E046EE50E069E670E081E090E00E9426
:10441000A404809138068330A9F4809136069091E7
:104420003706019790933706809336060FE110E028
:104430002CE330E046EE50E069E670E081E090E089
:104440000E94A40480913606909137064A9720F086
:10445000D0933706C0933606809136069091370682
:104460000A9720F4D0933706C0933606609136063B
:104470007091370688EB92E066C086EB92E00E946E
:104480008A447C0103E02FE130E040E058EF62E82D
:1044900070E080E590E00E94DF0586EB92E00E94EC
:1044A0008A4490931606809315060E94DD0C809135
:1044B00038068230A9F4809115069091160601966F
:1044C00090931606809315060FE110E02CE330E080
:1044D00046EE50E069E670E081E090E00E94A404BE
:1044E000809138068330A9F48091150690911606C4
:1044F000019790931606809315060FE110E02CE3C8
:1045000030E046EE50E069E670E081E090E00E9425
:10451000A40480911506909116064A9720F0D09336
:104520001606C093150680911506909116060A97F7
:1045300020F4D0931606C09315066091150670916D
:10454000160686EB92E00E94A5442FE788E391E0EF
:10455000215080409040E1F700C00000CBC084EBC8
:1045600092E00E948A447C0103E02FE130E040E0C9
:1045700058EF62E870E080E590E00E94DF0584EB90
:1045800092E00E948A4490933506809334060E94FC
:10459000DD0C809138068230A9F480913406909128
:1045A0003506019690933506809334060FE110E0AE
:1045B0002CE330E046EE50E069E670E081E090E008
:1045C0000E94A404809138068330A9F480913406B7
:1045D00090913506019790933506809334060FE14C
:1045E00010E02CE330E046EE50E069E670E081E058
:1045F00090E00E94A40480913406909135064F9774
:1046000020F0D0923506C092340680913406909105
:104610003506059720F4D0923506C0923406609195
:1046200034067091350684EB92E08DCF83EB92E0F7
:104630000E9482448093D9050E94DD0C8091380647
:10464000823089F48091D9058F5F8093D9050FE17D
:1046500010E02CE330E046EE50E069E670E081E0E7
:1046600090E00E94A40480913806833089F4809100
:10467000D90581508093D9050FE110E02CE330E09B
:1046800046EE50E069E670E081E090E00E94A4040C
:104690008091D905823010F01092D9058091D9050A
:1046A000813079F492E4E92E95E0F92E03E02FE1D0
:1046B00030E040E058EF62E870E080E590E00E9472
:1046C00099058091D90581110FC08DE3E82E85E011
:1046D000F82E03E02FE130E040E058EF62E870E0B0
:1046E00080E590E00E9499056091D90583EB92E006
:1046F0000E94984480913806813049F48093760670
:10470000809332068FE190E00E941906CCDCB092D3
:1047100038063BCEDF91CF911F910F91FF90EF9024
:10472000DF90CF90BF9008954F925F926F927F92EB
:104730008F929F92AF92BF92CF92DF92EF92FF92B1
:104740000F931F93CF93DF9380913306811163C141
:104750008FE190E00E9419060E94330B85E0809360
:1047600038061092320610922C0655245394C7E056
:10477000D0E0A6E0CA2ED12CB5E0AB2EB12C14E0CF
:10478000812E912C03E0602E712C85E0482E8091C3
:104790003306811140C10E94DD0C809138068230C1
:1047A00089F480912C068F5F80932C060FE110E036
:1047B0002CE330E046EE50E069E670E081E090E006
:1047C0000E94A40480913806833089F480912C06DD
:1047D000815080932C060FE110E02CE330E046EE90
:1047E00050E069E670E081E090E00E94A4048091CE
:1047F0002C06893010F010922C06E0912C068E2F9A
:1048000090E08930910508F0D4C0FC01E259FF4FD7
:104810000C946741FDE0EF2EF5E0FF2E02E02FE162
:1048200030E04FEF5FEF62E870E088E090E00E94D8
:104830009905109232061092130610921206B9C012
:10484000EFEFEE2EE4E0FE2E02E02FE130E04FEF3E
:104850005FEF68E770E088E090E00E9499051092B1
:10486000320681E090E013C071EFE72E74E0F72E7E
:1048700002E02FE130E04FEF5FEF68E770E088E0A3
:1048800090E00E9499051092320682E090E09093A9
:104890001306809312068DC065EEE62E64E0F62EB8
:1048A00002E02FE130E04FEF5FEF68E770E088E073
:1048B00090E00E9499051092320670921306609261
:1048C000120677C053EDE52E54E0F52E02E02FE1FD
:1048D00030E04FEF5FEF68E770E088E090E00E9423
:1048E000990510923206909213068092120661C0CA
:1048F0003DECE32E34E0F32E02E02FE130E04FEF09
:104900005FEF6EE670E088E290E00E94990543EC6C
:10491000E42E44E0F42E2FE130E04FEF5FEF67E844
:1049200070E08FE090E00E94990510923206B092FC
:104930001306A09212063DC026EBE22E24E0F22ED2
:1049400002E02FE130E04FEF5FEF68E770E088E0D2
:1049500090E00E94990510923206D0921306C09200
:10496000120627C098E9E92E94E0F92E02E02FE123
:1049700030E04FEF5FEF68E770E088E090E00E9482
:10498000990510923206D0931306C093120611C0F7
:1049900082EAE82E84E0F82E02E02FE130E04FEFCB
:1049A0005FEF68E770E082E090E00E949905509226
:1049B000320680913806813011F5809132068130BF
:1049C00059F41092130610921206109233068FE1DA
:1049D00090E00E94190667DB50923306109224067D
:1049E0001092230680911206909113069093000670
:1049F0008093FF058FE190E00E94190626DA40922D
:104A000038062FEF80E792E0215080409040E1F798
:104A100000C00000BCCEDF91CF911F910F91FF909D
:104A2000EF90DF90CF90BF90AF909F908F907F904E
:104A30006F905F904F900895EF92FF920F931F93A6
:104A4000CF93DF93A895809145068111F4C08FE143
:104A500090E00E9419060E944F0C80916E0690E033
:104A600090931E0680931D0685E080933806C1E072
:104A7000D5E0809145068111DEC0A8950E94DD0C2D
:104A8000809138068230A9F480911D0690911E060F
:104A9000019690931E0680931D060FE110E02CE313
:104AA00030E046EE50E069E670E081E090E00E9480
:104AB000A404809138068330A9F480911D0690915A
:104AC0001E06019790931E0680931D060FE110E0CD
:104AD0002CE330E046EE50E069E670E081E090E0E3
:104AE0000E94A40480911D0690911E06039720F059
:104AF00010921E0610921D0680911D0690911E06B2
:104B00008130910589F1D0F0029709F046C080E725
:104B1000E82E84E0F82E02E02FE130E04FEF5FEF67
:104B20006DE770E088E290E00E94990582E0809352
:104B30006E064EE150E06AE570E02BC024E8E22EFC
:104B400024E0F22E02E02FE130E04FEF5FEF6DE75F
:104B500070E088E290E00E94990510926E064EE1A6
:104B600050E066E970E015C09AE7E92E94E0F92E6E
:104B700002E02FE130E04FEF5FEF6DE770E088E299
:104B800090E00E949905C0936E064EE150E068E700
:104B900070E089EE95E00E947244809138068111A0
:104BA0000FC0A895C09345061092240610922306C4
:104BB000C09333068FE190E00E941906A89545D96D
:104BC00080913806813059F5A8958093450610925A
:104BD000240610922306809333068FE190E00E9412
:104BE0001906A89510927D0680916E06813069F0B5
:104BF00038F0823091F44EE150E06AE570E009C08F
:104C00004EE150E066E970E004C04EE150E068E734
:104C100070E089EE95E00E947244A89513D0D0937D
:104C200038062FEF80E792E0215080409040E1F776
:104C300000C000001ECFDF91CF911F910F91FF9018
:104C4000EF900895EF92FF920F931F93CF9380916F
:104C50007D0681110C9426318FE190E00E941906A7
:104C60000E94450D85E080933806C5E080917D0661
:104C700081110C9426310E94DD0C8091380682301F
:104C8000D9F4809169068F5F809369060FE110E087
:104C90002CE330E046EE50E069E670E081E090E021
:104CA0000E94A40422E330E043EC50E068E270E0AC
:104CB00088E090E00E94A404809138068330D9F403
:104CC000809169068150809369060FE110E02CE322
:104CD00030E046EE50E069E670E081E090E00E944E
:104CE000A40422E330E043EC50E068E270E088E0A6
:104CF00090E00E94A404809169068E3010F010921A
:104D00006906E09169068E2F90E08E30910510F0D3
:104D10000C94C92FFC01E958FF4F80911206909125
:104D200013060C946741892BB9F58091E9059091A0
:104D3000EA05893E934020F01092EA051092E905B9
:104D40007AE2E72E74E0F72E01E02FE130E04FEF3A
:104D50005FEF62E370E08FE090E00E949905E3E28C
:104D6000EE2EE4E0FE2E2FE130E04FEF5FEF66E441
:104D700070E08CE390E00E949905E090E905F090E6
:104D8000EA0503E02FE130E04FEF5FEF62E870E00B
:104D900080E590E00E94DF05809112069091130655
:104DA000019709F0F1C78091E9059091EA05893EE4
:104DB000934020F01092EA051092E9055AE2E52EA0
:104DC00054E0F52E01E02FE130E04FEF5FEF62E3BA
:104DD00070E08FE090E00E94990563E2E62E64E0C7
:104DE000F62E2FE130E04FEF5FEF66E470E08CE3EA
:104DF00090E00E949905E090E905F090EA05B9C7B6
:104E0000892BB9F58091EB059091EC05893E934093
:104E100020F01092EC051092EB053BE0E32E34E01D
:104E2000F32E01E02FE130E04FEF5FEF62E370E03F
:104E30008FE090E00E9499054DEFE42E43E0F42EC0
:104E40002FE130E04FEF5FEF66E470E08CE390E03D
:104E50000E949905E090EB05F090EC0503E02FE14E
:104E600030E04FEF5FEF62E870E080E590E00E9495
:104E7000DF0580911206909113068130910531F47F
:104E8000809169068F5F8093690639C00297B9F5F2
:104E90008091EB059091EC05893E934020F01092B3
:104EA000EC051092EB059BE0E92E94E0F92E01E071
:104EB0002FE130E04FEF5FEF62E370E08FE090E0D2
:104EC0000E9499052DEFE22E23E0F22E2FE130E033
:104ED0004FEF5FEF66E470E08CE390E00E9499058D
:104EE000E090EB05F090EC0503E02FE130E04FEFB0
:104EF0005FEF62E870E080E590E00E94DF0580915E
:104F00001206909113060497B9F58091EB059091E4
:104F1000EC05893E934020F01092EC051092EB05D1
:104F20000BE0E02E04E0F02E01E02FE130E04FEF47
:104F30005FEF62E370E08FE090E00E9499058DEFF3
:104F4000E82E83E0F82E2FE130E04FEF5FEF66E4CC
:104F500070E08CE390E00E949905E090EB05F09002
:104F6000EC0503E02FE130E04FEF5FEF62E870E027
:104F700080E590E00E94DF05809112069091130673
:104F80000597B9F58091EB059091EC05893E93402A
:104F900020F01092EC051092EB05BBE0EB2EB4E094
:104FA000FB2E01E02FE130E04FEF5FEF62E370E0B6
:104FB0008FE090E00E9499051DEFE12E13E0F12EA5
:104FC0002FE130E04FEF5FEF66E470E08CE390E0BC
:104FD0000E949905E090EB05F090EC0503E02FE1CD
:104FE00030E04FEF5FEF62E870E080E590E00E9414
:104FF000DF058091120690911306069709F0C9C744
:105000008091EB059091EC05893E934020F0109241
:10501000EC051092EB05FBE0EF2EF4E0FF2E01E033
:105020002FE130E04FEF5FEF62E370E08FE090E060
:105030000E949905ADEFEA2EA3E0FA2E2FE130E0B1
:105040004FEF5FEF66E470E08CE390E00E9499051B
:10505000E090EB05F090EC05E0C5892BB1F580916F
:10506000ED059091EE054F9720F01092EE0510920D
:10507000ED0575EEE72E73E0F72E01E02FE130E04D
:105080004FEF5FEF62E370E08FE090E00E949905E0
:10509000EDECEE2EE3E0FE2E2FE130E04FEF5FEF80
:1050A00066E470E08FE090E00E949905E090ED05E5
:1050B000F090EE0503E02FE130E04FEF5FEF62E8A4
:1050C00070E080E590E00E94DF05809112069091EB
:1050D0001306019709F058C68091ED059091EE05F1
:1050E0004F9720F01092EE051092ED0555EEE52E4B
:1050F00053E0F52E01E02FE130E04FEF5FEF62E388
:1051000070E08FE090E00E9499056DECE62E63E080
:10511000F62E2FE130E04FEF5FEF66E470E08FE0B6
:1051200090E00E949905E090ED05F090EE0521C613
:10513000892BB1F58091EF059091F0054F9720F004
:105140001092F0051092EF0535EBE32E33E0F32ECD
:1051500001E02FE130E04FEF5FEF62E370E08FE0BE
:1051600090E00E9499054DE9E42E43E0F42E2FE1F2
:1051700030E04FEF5FEF66E470E08FE090E00E9478
:105180009905E090EF05F090F00503E02FE130E0A5
:105190004FEF5FEF62E870E080E590E00E94DF058E
:1051A00080911206909113068130910531F480911F
:1051B00069068F5F8093690638C00297B1F58091C8
:1051C000EF059091F0054F9720F01092F0051092A6
:1051D000EF0595EBE92E93E0F92E01E02FE130E0A9
:1051E0004FEF5FEF62E370E08FE090E00E9499057F
:1051F0002DE9E22E23E0F22E2FE130E04FEF5FEFBA
:1052000066E470E08FE090E00E949905E090EF0581
:10521000F090F00503E02FE130E04FEF5FEF62E840
:1052200070E080E590E00E94DF0580911206909189
:1052300013060497B1F58091EF059091F0054F9713
:1052400020F01092F0051092EF0505EBE02E03E040
:10525000F02E01E02FE130E04FEF5FEF62E370E00E
:105260008FE090E00E9499058DE9E82E83E0F82E0A
:105270002FE130E04FEF5FEF66E470E08FE090E009
:105280000E949905E090EF05F090F00503E02FE112
:1052900030E04FEF5FEF62E870E080E590E00E9461
:1052A000DF0580911206909113060597B1F5809164
:1052B000EF059091F0054F9720F01092F0051092B5
:1052C000EF05B5EBEB2EB3E0FB2E01E02FE130E074
:1052D0004FEF5FEF62E370E08FE090E00E9499058E
:1052E0001DE9E12E13E0F12E2FE130E04FEF5FEFEB
:1052F00066E470E08FE090E00E949905E090EF0591
:10530000F090F00503E02FE130E04FEF5FEF62E84F
:1053100070E080E590E00E94DF0580911206909198
:105320001306069709F035C68091EF059091F005B8
:105330004F9720F01092F0051092EF05F5EBEF2E4D
:10534000F3E0FF2E01E02FE130E04FEF5FEF62E38B
:1053500070E08FE090E00E949905ADE9EA2EA3E0AD
:10536000FA2E2FE130E04FEF5FEF66E470E08FE060
:1053700090E00E949905E090EF05F090F0054DC493
:10538000892B09F045C08091F1059091F2050397B2
:1053900030F081E090E09093F2058093F105E5E82C
:1053A000EE2EE3E0FE2E01E02FE130E04FEF5FEF65
:1053B0006CE370E08FE090E00E9499058091F10528
:1053C0009091F205019779F472E4E72E75E0F72EDB
:1053D00003E02FE130E04FEF5FEF62E870E080E53F
:1053E00090E00E9499058091F1059091F205892B3A
:1053F00079F46DE3E62E65E0F62E03E02FE130E070
:105400004FEF5FEF62E870E080E590E00E94990561
:1054100080911206909113068130910509F044C0E5
:105420002091F1053091F2052330310520F0909361
:10543000F2058093F10555E8E52E53E0F52E01E0E5
:105440002FE130E04FEF5FEF6CE370E08FE090E032
:105450000E9499058091F1059091F205019779F4E8
:1054600042E4E42E45E0F42E03E02FE130E04FEF7C
:105470005FEF62E870E080E590E00E94990580911E
:10548000F1059091F205892B79F43DE3E32E35E0A7
:10549000F32E03E02FE130E04FEF5FEF62E870E0C2
:1054A00080E590E00E949905809112069091130684
:1054B000029709F045C08091F1059091F20503979C
:1054C00030F081E090E09093F2058093F10525E8BB
:1054D000E22E23E0F22E01E02FE130E04FEF5FEF0C
:1054E0006CE370E08FE090E00E9499058091F105F7
:1054F0009091F205019779F492E4E92E95E0F92E66
:1055000003E02FE130E04FEF5FEF62E870E080E50D
:1055100090E00E9499058091F1059091F205892B08
:1055200079F48DE3E82E85E0F82E03E02FE130E0FA
:105530004FEF5FEF62E870E080E590E00E94990530
:1055400080911206909113069C012450310922305B
:10555000310508F4D9C4069709F01BC58091F105FF
:105560009091F205039730F081E090E09093F2057E
:105570008093F10505E8E02E03E0F02E01E02FE135
:1055800030E04FEF5FEF6CE370E08FE090E00E945F
:1055900099058091F1059091F205019779F412E453
:1055A000E12E15E0F12E03E02FE130E04FEF5FEF49
:1055B00062E870E080E590E00E9499058091F10535
:1055C0009091F205892B09F0E4C4BDE3EB2EB5E020
:1055D000FB2E03E02FE130E04FEF5FEF62E870E079
:1055E00080E590E00E949905D4C4892BB9F580919B
:1055F000F3059091F4058F35914020F01092F40559
:105600001092F305FDE6EF2EF3E0FF2E01E02FE10F
:1056100030E04FEF5FEF62E370E08FE090E00E94D8
:105620009905A5E5EA2EA3E0FA2E2FE130E04FEF31
:105630005FEF66E470E08FE090E00E949905E090F3
:10564000F305F090F40503E02FE130E04FEF5FEF5A
:1056500062E870E080E590E00E94DF05809112062C
:10566000909113060197B9F58091F3059091F40597
:105670008F35914020F01092F4051092F3057DE6ED
:10568000E72E73E0F72E01E02FE130E04FEF5FEF00
:1056900062E370E08FE090E00E949905E5E5EE2E70
:1056A000E3E0FE2E2FE130E04FEF5FEF66E470E0C5
:1056B0008FE090E00E949905E090F305F090F405EA
:1056C00003E02FE130E04FEF5FEF62E870E080E54C
:1056D00090E00E94DF0580911206909113060297D8
:1056E000B9F58091F3059091F4058F35914020F044
:1056F0001092F4051092F3055DE6E52E53E0F52EC9
:1057000001E02FE130E04FEF5FEF62E370E08FE008
:1057100090E00E94990565E5E62E63E0F62E2FE104
:1057200030E04FEF5FEF66E470E08FE090E00E94C2
:105730009905E090F305F090F40503E02FE130E0E7
:105740004FEF5FEF62E870E080E590E00E94DF05D8
:1057500080911206909113069C0124503109223049
:10576000310508F4D1C3069709F013C48091F305FD
:105770009091F4058F35914020F01092F40510922D
:10578000F3053DE6E32E33E0F32E01E02FE130E0B8
:105790004FEF5FEF62E370E08FE090E00E949905C9
:1057A00045E5E42E43E0F42E2FE130E04FEF5FEFCC
:1057B00066E470E08FE090E00E949905E090F305C8
:1057C000F090F4052AC2892BB9F58091F5059091E6
:1057D000F6058636910520F01092F6051092F50533
:1057E0009DE3E92E93E0F92E01E02FE130E04FEF49
:1057F0005FEF62E370E08FE090E00E94990525E2A0
:10580000E22E23E0F22E2FE130E04FEF5FEF66E46F
:1058100070E08FE090E00E949905E090F505F0902F
:10582000F60503E02FE130E04FEF5FEF62E870E054
:1058300080E590E00E94DF058091120690911306AA
:105840000197B9F58091F5059091F6058636910599
:1058500020F01092F6051092F5050DE3E02E03E01E
:10586000F02E01E02FE130E04FEF5FEF62E370E0F8
:105870008FE090E00E94990585E2E82E83E0F82E03
:105880002FE130E04FEF5FEF66E470E08FE090E0F3
:105890000E949905E090F505F090F60503E02FE1F0
:1058A00030E04FEF5FEF62E870E080E590E00E944B
:1058B000DF0580911206909113068230910531F434
:1058C000809169068F5F8093690639C00497B9F5A6
:1058D0008091F5059091F6058636910520F010929D
:1058E000F6051092F505BDE3EB2EB3E0FB2E01E0CB
:1058F0002FE130E04FEF5FEF62E370E08FE090E088
:105900000E94990515E2E12E13E0F12E2FE130E01F
:105910004FEF5FEF66E470E08FE090E00E94990542
:10592000E090F505F090F60503E02FE130E04FEF51
:105930005FEF62E870E080E590E00E94DF05809113
:105940001206909113060597B9F58091F50590918F
:10595000F6058636910520F01092F6051092F505B1
:10596000FDE3EF2EF3E0FF2E01E02FE130E04FEFFB
:105970005FEF62E370E08FE090E00E949905A5E29E
:10598000EA2EA3E0FA2E2FE130E04FEF5FEF66E45E
:1059900070E08FE090E00E949905E090F505F090AE
:1059A000F60503E02FE130E04FEF5FEF62E870E0D3
:1059B00080E590E00E94DF05809112069091130629
:1059C000A0C2892BB9F58091F7059091F80586362C
:1059D000910520F01092F8051092F7057DE0E72E72
:1059E00073E0F72E01E02FE130E04FEF5FEF62E36D
:1059F00070E08FE090E00E949905E5EFEE2EE2E086
:105A0000FE2E2FE130E04FEF5FEF66E470E08FE0B5
:105A100090E00E949905E090F705F090F80503E00A
:105A20002FE130E04FEF5FEF62E870E080E590E05B
:105A30000E94DF0580911206909113068130910536
:105A400031F4809169068F5F8093690639C00297AF
:105A5000B9F58091F7059091F8058636910520F00B
:105A60001092F8051092F7055DE0E52E53E0F52E53
:105A700001E02FE130E04FEF5FEF62E370E08FE095
:105A800090E00E94990565EFE62E62E0F62E2FE188
:105A900030E04FEF5FEF66E470E08FE090E00E944F
:105AA0009905E090F705F090F80503E02FE130E06C
:105AB0004FEF5FEF62E870E080E590E00E94DF0565
:105AC00080911206909113060497B9F58091F7051D
:105AD0009091F8058636910520F01092F805109205
:105AE000F7053DE0E32E33E0F32E01E02FE130E057
:105AF0004FEF5FEF62E370E08FE090E00E94990566
:105B000045EFE42E42E0F42E2FE130E04FEF5FEF5F
:105B100066E470E08FE090E00E949905E090F70560
:105B2000F090F80503E02FE130E04FEF5FEF62E81F
:105B300070E080E590E00E94DF0580911206909170
:105B400013060597B9F58091F7059091F80586360B
:105B5000910520F01092F8051092F7059DE0E92ECE
:105B600093E0F92E01E02FE130E04FEF5FEF62E3C9
:105B700070E08FE090E00E94990525EFE22E22E090
:105B8000F22E2FE130E04FEF5FEF66E470E08FE040
:105B900090E00E949905E090F705F090F80503E089
:105BA0002FE130E04FEF5FEF62E870E080E590E0DA
:105BB0000E94DF058091120690911306069709F066
:105BC000E8C18091F7059091F8058636910520F09F
:105BD0001092F8051092F7051DE0E12E13E0F12E6A
:105BE00001E02FE130E04FEF5FEF62E370E08FE024
:105BF00090E00E94990585EFE82E82E0F82E2FE1D3
:105C000030E04FEF5FEF66E470E08FE090E00E94DD
:105C10009905E090F705F090F80503E02FE130E0FA
:105C20004FEF5FEF62E870E080E590E00E94DF05F3
:105C3000B0C1892B49F580910106909102068D3201
:105C4000914020F01092020610920106B5E7EB2E6B
:105C5000B2E0FB2E01E02FE130E04FEF5FEF6CE3AD
:105C600070E08FE090E00E949905E0900106F090CE
:105C7000020603E02FE130E04FEF5FEF62E870E0F3
:105C800080E590E00E94DF05809112069091130656
:105C9000019709F079C080910106909102068D323A
:105CA000914020F01092020610920106A5E7EA2E1C
:105CB000A2E0FA2E01E02FE130E04FEF5FEF6CE35E
:105CC00070E08FE090E00E949905E0900106F0906E
:105CD00002064FC0892B49F5809103069091040676
:105CE000893E934020F01092040610920306FBECCC
:105CF000EF2EF2E0FF2E01E02FE130E04FEF5FEFFB
:105D00006CE370E08FE090E00E949905E09003065C
:105D1000F090040603E02FE130E04FEF5FEF62E820
:105D200070E080E590E00E94DF058091120690917E
:105D30001306019749F58091030690910406893E68
:105D4000934020F01092040610920306EBECEE2E26
:105D5000E2E0FE2E01E02FE130E04FEF5FEF6CE379
:105D600070E08FE090E00E949905E0900306F090CB
:105D7000040603E02FE130E04FEF5FEF62E870E0F0
:105D800080E590E00E94DF05809112069091130655
:105D90008230910509F4B8C09C01245031092230A9
:105DA000310508F0AEC0B0C0892B09F094C08091D5
:105DB000F9059091FA05039720F01092FA051092D8
:105DC000F90573EEE72E72E0F72E01E02FE130E0E7
:105DD0004FEF5FEF6CE370E08EE190E00E94990579
:105DE0008091F9059091FA05019779F462E4E62E25
:105DF00065E0F62E03E02FE130E04FEF5FEF62E861
:105E000070E080E590E00E9499058091F9059091FD
:105E1000FA05892B79F45DE3E52E55E0F52E03E0D4
:105E20002FE130E04FEF5FEF62E870E080E590E057
:105E30000E9499058091F9058093D8054CC0892B63
:105E400009F049C08091D80581110BC010926906F4
:105E500053C0892B09F03FC08091D805811149C0FA
:105E6000F5CF813009F048C08091FB059091FC0589
:105E7000893E934020F01092FC051092FB053DE610
:105E8000E32E33E0F32E01E02FE130E04FEF5FEF40
:105E900062E370E08FE090E00E94990545EBE42E0C
:105EA00042E0F42E2FE130E04FEF5FEF66E470E068
:105EB0008FE090E00E949905E090FB05F090FC05D2
:105EC00003E02FE130E04FEF5FEF62E870E080E544
:105ED00090E00E94DF0580911206909113068130B8
:105EE000910591F08230910579F08430910561F04F
:105EF00005C0813009F47DC180E090E085309105D6
:105F000019F0069709F045C0809169068F5F80936C
:105F100069063FC0009731F09C01215031092230C1
:105F2000310518F4109269062BC0049749F5809149
:105F3000050690910606893E934020F010920606D1
:105F4000109205068EE4E82E82E0F82E01E02FE1A3
:105F500030E04FEF5FEF6CE370E08FE090E00E9485
:105F60009905E0900506F090060603E02FE130E089
:105F70004FEF5FEF62E870E080E590E00E94DF05A0
:105F800080911206909113060597029710F41092D3
:105F9000690680913806813009F00EC180937D0634
:105FA000109245068091120690911306892B41F5B7
:105FB000E0911D06F0911E06E830F10508F5EB575B
:105FC000FF4F4EE150E00C94674164E972E014C069
:105FD00066E772E011C068E572E00EC06AE372E045
:105FE0000BC06CE172E008C06EEF71E005C060EEBE
:105FF00071E002C062EC71E089EE95E00E948F448E
:1060000080911206909113060197E1F480911D068C
:1060100090911E068130910569F038F0029791F455
:106020004EE150E068E671E009C04EE150E064EAFC
:1060300071E004C04EE150E066E871E089EE95E061
:106040000E948F4480911206909113060297E1F40A
:1060500080911D0690911E068130910569F038F0FF
:10606000029791F44EE150E06EE071E009C04EE11C
:1060700050E06AE471E004C04EE150E06CE271E08F
:1060800089EE95E00E948F4480911206909113064C
:106090000497E1F480911D0690911E0681309105D0
:1060A00069F038F0029791F44EE150E064EB70E053
:1060B00009C04EE150E060EF70E004C04EE150E0F6
:1060C00062ED70E089EE95E00E948F4480911206A7
:1060D000909113060597E1F480911D0690911E069C
:1060E0008130910569F038F0029791F44EE150E06B
:1060F0006AE570E009C04EE150E066E970E004C076
:106100004EE150E068E770E089EE95E00E948F4430
:1061100080911206909113060697E1F480911D0676
:1061200090911E068130910569F038F0029791F444
:106130004EE150E060E070E009C04EE150E06CE3F9
:1061400070E004C04EE150E06EE170E089EE95E051
:106150000E948F448FE190E00E9419068091120600
:1061600090911306892B09F47FD1809112069091AA
:106170001306019711F40E94D03A80911206909173
:106180001306029711F40E94D73B8091120690915A
:106190001306049711F40E94DC3C80911206909142
:1061A0001306059711F40E941C2580911206909108
:1061B0001306069709F450D08091380681110CC05F
:1061C00081E080937D0610924506109207068FE1CC
:1061D00090E00E941906EBD2C09338068FE798E34F
:1061E00021E0815090402040E1F700C000000C9475
:1061F00036268091FD059091FE05893E934020F062
:106200001092FE051092FD059EE9E92E92E0F92E0E
:1062100001E02FE130E04FEF5FEF62E370E08FE0ED
:1062200090E00E9499052BE8E22E22E0F22E2FE169
:1062300030E04FEF5FEF66E470E08FE090E00E94A7
:106240009905E090FD05F090FE053ACECF911F91A3
:106250000F91FF90EF900895EF92FF920F931F938D
:10626000CF93DF93A895809145068111F6C08FE109
:1062700090E00E9419060E944F0C80916B0690E0FE
:1062800090931E0680931D0685E080933806C1E03A
:10629000D5E0809145068111E0C0A8950E94DD0CF3
:1062A000809138068230A9F480911D0690911E06D7
:1062B000019690931E0680931D060FE110E02CE3DB
:1062C00030E046EE50E069E670E081E090E00E9448
:1062D000A404809138068330A9F480911D06909122
:1062E0001E06019790931E0680931D060FE110E095
:1062F0002CE330E046EE50E069E670E081E090E0AB
:106300000E94A40480911D0690911E06039720F020
:1063100010921E0610921D0680911D0690911E0679
:106320008130910589F1D0F0029709F046C080E7ED
:10633000E82E84E0F82E02E02FE130E04FEF5FEF2F
:106340006DE770E088E290E00E94990582E080931A
:106350006B064EE150E060E070E02BC024E8E22ED6
:1063600024E0F22E02E02FE130E04FEF5FEF6DE727
:1063700070E088E290E00E94990510926B064EE171
:1063800050E06CE370E015C09AE7E92E94E0F92E36
:1063900002E02FE130E04FEF5FEF6DE770E088E261
:1063A00090E00E949905C0936B064EE150E06EE1CB
:1063B00070E089EE95E00E94724480913806811168
:1063C00010C0A895C093450610922406109223068B
:1063D000C09333068FE190E00E941906A8950E94B1
:1063E000251F80913806813061F5A8958093450678
:1063F0001092240610922306809333068FE190E0DA
:106400000E941906A89510927D0680916B06813036
:1064100069F038F0823091F44EE150E060E070E0D5
:1064200009C04EE150E06CE370E004C04EE150E082
:106430006EE170E089EE95E00E947244A8950E949A
:106440002226D09338062FEF80E792E0215080403B
:106450009040E1F700C000001CCFDF91CF911F9169
:106460000F91FF90EF900895AF92BF92CF92DF927D
:10647000EF92FF920F931F93CF93DF93A895809194
:106480004506811189C18FE190E00E9419060E94A2
:106490004F0C80916F0690E090931E0680931D062E
:1064A00085E080933806E7E0DE2EF6E0CF2ED5E0DB
:1064B000A4E0BA2EB3E0AB2EC1E080914506811175
:1064C0006BC1A8950E94DD0C809138068230A9F43A
:1064D00080911D0690911E06019690931E06809352
:1064E0001D060FE110E02CE330E046EE50E069E6D7
:1064F00070E081E090E00E94A4048091380683302F
:10650000A9F480911D0690911E06019790931E0696
:1065100080931D060FE110E02CE330E046EE50E0E2
:1065200069E670E081E090E00E94A40480911D067D
:1065300090911E06089720F010921E0610921D06DC
:10654000E0911D06F0911E06E830F10508F0BEC08E
:10655000E357FF4F0C94674173E9E72E74E0F72E81
:1065600002E02FE130E04FEF5FEF6DE770E082E394
:1065700090E00E94990510926F064EE150E064E9A8
:1065800072E09AC06EE8E62E64E0F62E02E02FE19B
:1065900030E04FEF5FEF6DE770E082E390E00E9444
:1065A0009905C0936F064EE150E066E772E084C043
:1065B00054E8E52E54E0F52E02E02FE130E04FEFF5
:1065C0005FEF6DE770E088E290E00E94990582E05D
:1065D00080936F064EE150E068E572E06DC04AE7D7
:1065E000E42E44E0F42E02E02FE130E04FEF5FEFC5
:1065F0006DE770E088E290E00E949905A0926F0636
:106600004EE150E06AE372E057C030E7E32E34E039
:10661000F32E02E02FE130E04FEF5FEF6DE770E027
:1066200088E290E00E949905B0926F0644E150E044
:106630006CE172E041C026E6E22E24E0F22E02E098
:106640002FE130E04FEF5FEF6DE770E088E290E020
:106650000E949905D0936F064EE150E06EEF71E015
:106660002BC09CE5E92E94E0F92E02E02FE130E00A
:106670004FEF5FEF6DE770E088E290E00E949905D0
:10668000C0926F064EE150E060EE71E015C082E509
:10669000E82E84E0F82E02E02FE130E04FEF5FEFCC
:1066A0006DE770E088E290E00E949905D0926F0655
:1066B0004EE150E062EC71E089EE95E00E94724498
:1066C0008FE59AEE0197F1F700C00000809138063F
:1066D00081110FC0A895C093450610922406109210
:1066E0002306C09333068FE190E00E9419060E94B2
:1066F000251F80913806813009F041C0A89580930C
:1067000045061092240610922306809333068FE1EB
:1067100090E00E94190610927D06E0916F068E2F80
:1067200090E08830910540F5FC01EB56FF4F4EE1BB
:1067300050E00C94674164E972E014C066E772E0CF
:1067400011C068E572E00EC06AE372E00BC06CE154
:1067500072E008C06EEF71E005C060EE71E002C04B
:1067600062EC71E089EE95E00E9472448FE59AEE4A
:106770000197F1F700C00000A8950E942226D0934F
:106780003806A8959FEF20E782E091502040804096
:10679000E1F700C0000091CEDF91CF911F910F91E2
:1067A000FF90EF90DF90CF90BF90AF900895BF9291
:1067B000CF92DF92EF92FF920F931F93CF93DF93CD
:1067C000809107068111E2C68FE190E00E941906D0
:1067D0000E94450D10926A0685E08093380698E580
:1067E000C92E92E0D92ECAE5D0E025E0B22E8091E4
:1067F00007068111CBC6E09169068E2F90E08E309E
:10680000910508F0B2C6FC01E356FF4F0C946741B6
:106810001AE2E12E14E0F12E01E02FE130E04FEF1B
:106820005FEF62E370E08FE090E00E94990583E201
:10683000E82E84E0F82E2FE130E04FEF5FEF66E4C2
:1068400070E08CE390E00E949905E090E905F090FB
:10685000EA0503E02FE130E040E058EF62E870E045
:1068600080E590E00E94DF058091E9059091EA05BE
:106870009093DD058093DC050E94DD0C8091380645
:106880008230A9F48091DC059091DD05019690930A
:10689000DD058093DC050FE110E02CE330E046EEEF
:1068A00050E069E670E081E090E00E94A4048091ED
:1068B00038068330A9F48091DC059091DD050197BD
:1068C0009093DD058093DC050FE110E02CE330E0D0
:1068D00046EE50E069E670E081E090E00E94A4049A
:1068E0008091DC059091DD058F35914020F010926C
:1068F000DD051092DC058091DC059091DD0590931B
:10690000EA058093E90528C6ABE0EA2EA4E0FA2E5A
:1069100001E02FE130E04FEF5FEF62E370E08FE0E6
:1069200090E00E949905BDEFEB2EB3E0FB2E2FE126
:1069300030E04FEF5FEF66E470E08CE390E00E94A0
:106940009905E090EB05F090EC0503E02FE130E0D5
:1069500040E058EF62E870E080E590E00E94DF05DB
:106960008091EB059091EC059093300680932F0673
:106970000E94DD0C809138068230A9F480912F06A8
:106980009091300601969093300680932F060FE188
:1069900010E02CE330E046EE50E069E670E081E084
:1069A00090E00E94A404809138068330A9F480917D
:1069B0002F069091300601979093300680932F0612
:1069C0000FE110E02CE330E046EE50E069E670E0C5
:1069D00081E090E00E94A40480912F0690913006FF
:1069E000853F914020F01092300610922F06809142
:1069F0002F06909130069093EC058093EB05ACC583
:106A0000E5EEEE2EE3E0FE2E01E02FE130E04FEF69
:106A10005FEF62E370E08FE090E00E949905FDEC8B
:106A2000EF2EF3E0FF2E2FE130E04FEF5FEF66E453
:106A300070E08FE090E00E949905E090ED05F09005
:106A4000EE0503E02FE130E040E058EF62E870E04F
:106A500080E590E00E94DF058091ED059091EE05C4
:106A600090937806809377060E94DD0C809138061B
:106A70008230A9F4809177069091780601969093E0
:106A80007806809377060FE110E02CE330E046EEC5
:106A900050E069E670E081E090E00E94A4048091FB
:106AA00038068330A9F48091770690917806019793
:106AB00090937806809377060FE110E02CE330E0A6
:106AC00046EE50E069E670E081E090E00E94A404A8
:106AD00080917706909178064F9730F08FE090E0A4
:106AE0009093780680937706809177069091780648
:106AF0000F9730F48FE090E09093780680937706BC
:106B000080917706909178069093EE058093ED053D
:106B100023C565EBE62E63E0F62E01E02FE130E0C1
:106B20004FEF5FEF62E370E08FE090E00E94990525
:106B30007DE9E72E73E0F72E2FE130E04FEF5FEFB6
:106B400066E470E08FE090E00E949905E090EF0528
:106B5000F090F00503E02FE130E040E058EF62E80C
:106B600070E080E590E00E94DF058091EF05909154
:106B7000F00590931A06809319060E94DD0C80910F
:106B800038068230A9F48091190690911A06019670
:106B900090931A06809319060FE110E02CE330E081
:106BA00046EE50E069E670E081E090E00E94A404C7
:106BB000809138068330A9F48091190690911A06C5
:106BC000019790931A06809319060FE110E02CE3C9
:106BD00030E046EE50E069E670E081E090E00E942F
:106BE000A4048091190690911A064F9730F08FE017
:106BF00090E090931A06809319068091190690915F
:106C00001A060F9730F48FE090E090931A06809365
:106C100019068091190690911A069093F0058093B9
:106C2000EF059AC455E8E52E53E0F52E01E02FE17B
:106C300030E04FEF5FEF6CE370E08FE090E00E9498
:106C400099058091F1059091F205019779F442E45C
:106C5000E42E45E0F42E03E02FE130E040E058EF71
:106C600062E870E080E590E00E9499058091F1056E
:106C70009091F205892B79F43DE3E32E35E0F32E74
:106C800003E02FE130E040E058EF62E870E080E59B
:106C900090E00E9499058091F105809344060E943E
:106CA000DD0C80913806823089F4809144068F5F34
:106CB000809344060FE110E02CE330E046EE50E014
:106CC00069E670E081E090E00E94A40480913806BB
:106CD000833089F4809144068150809344060FE10B
:106CE00010E02CE330E046EE50E069E670E081E031
:106CF00090E00E94A40480914406823010F010922B
:106D000044068091440690E09093F2058093F1054B
:106D100023C49DE6E92E93E0F92E01E02FE130E057
:106D20004FEF5FEF62E370E08FE090E00E94990523
:106D300025E5E22E23E0F22E2FE130E04FEF5FEF6A
:106D400066E470E08FE090E00E949905E090F30522
:106D5000F090F40503E020E038EF4FEF5FEF62E8DA
:106D600070E080E590E00E94DF058091F30590914E
:106D7000F40590931806809317060E94DD0C80910D
:106D800038068230A9F48091170690911806019672
:106D900090931806809317060FE110E02CE330E083
:106DA00046EE50E069E670E081E090E00E94A404C5
:106DB000809138068330A9F48091170690911806C7
:106DC000019790931806809317060FE110E02CE3CB
:106DD00030E046EE50E069E670E081E090E00E942D
:106DE000A40480911706909118068B3F910520F01E
:106DF00010921806109217068091170690911806A7
:106E00009093F4058093F305A7C31DE3E12E13E0EF
:106E1000F12E01E02FE130E04FEF5FEF62E370E031
:106E20008FE090E00E94990585E2E82E83E0F82E3D
:106E30002FE130E04FEF5FEF66E470E08FE090E02D
:106E40000E949905E090F505F090F60503E02FE12A
:106E500030E040E058EF62E870E080E590E00E94AA
:106E6000DF058091F505809328060E94DD0C809156
:106E70003806823089F4809128068F5F8093280637
:106E80000FE110E02CE330E046EE50E069E670E000
:106E900081E090E00E94A40480913806833089F458
:106EA000809128068150809328060FE110E02CE3A2
:106EB00030E046EE50E069E670E081E090E00E944C
:106EC000A40480912806853610F01092280680913F
:106ED000280690E09093F6058093F5053DC3ADE05C
:106EE000EA2EA3E0FA2E01E02FE130E04FEF5FEF52
:106EF00062E370E08FE090E00E949905B5EFEB2E21
:106F0000B2E0FB2E2FE130E04FEF5FEF66E470E080
:106F10008FE090E00E949905E090F705F090F80569
:106F200003E02FE130E040E058EF62E870E080E5F8
:106F300090E00E94DF058091F705809327060E946C
:106F4000DD0C80913806823089F4809127068F5FAE
:106F5000809327060FE110E02CE330E046EE50E08E
:106F600069E670E081E090E00E94A4048091380618
:106F7000833089F4809127068150809327060FE1A2
:106F800010E02CE330E046EE50E069E670E081E08E
:106F900090E00E94A40480912706853610F010929C
:106FA00027068091270690E09093F8058093F705D7
:106FB000D3C2F5E7EF2EF2E0FF2E01E02FE130E043
:106FC0004FEF5FEF6CE370E08FE090E00E94990577
:106FD000E0900106F090020603E02FE130E040E08F
:106FE00058EF62E870E080E590E00E94DF05809154
:106FF00001069091020690936606809365060E94B2
:10700000DD0C809138068230A9F48091650690915C
:107010006606019690936606809365060FE110E080
:107020002CE330E046EE50E069E670E081E090E06D
:107030000E94A404809138068330A9F480916506EB
:1070400090916606019790936606809365060FE11E
:1070500010E02CE330E046EE50E069E670E081E0BD
:1070600090E00E94A4048091650690916606893C98
:10707000910520F0D0936606C09365068091650661
:10708000909166068A35910520F4D0936606C093E8
:10709000650680916506909166069093020680933E
:1070A00001065AC2EBECEE2EE2E0FE2E01E02FE1EB
:1070B00030E04FEF5FEF6CE370E08FE090E00E9414
:1070C0009905E0900306F090040603E02FE130E01C
:1070D00040E058EF62E870E080E590E00E94DF0554
:1070E00080910306909104069093E8058093E7054C
:1070F0000E94DD0C809138068230A9F48091E7056A
:107100009091E80501969093E8058093E7050FE1DB
:1071100010E02CE330E046EE50E069E670E081E0FC
:1071200090E00E94A404809138068330A9F48091F5
:10713000E7059091E80501979093E8058093E705AE
:107140000FE110E02CE330E046EE50E069E670E03D
:1071500081E090E00E94A4048091E7059091E80509
:10716000C39720F01092E8051092E7058091E7059B
:107170009091E8059093040680930306EDC173EEA9
:10718000E72E72E0F72E01E02FE130E04FEF5FEFE6
:107190006CE370E08EE190E00E9499058091F90522
:1071A0009091FA05019779F462E4E62E65E0F62EF7
:1071B00003E02FE130E040E058EF62E870E080E566
:1071C00090E00E9499058091F9059091FA05892B2C
:1071D00079F45DE3E52E55E0F52E03E02FE130E094
:1071E00040E058EF62E870E080E590E00E94990589
:1071F0008091F9058093D8050E94DD0C80913806B6
:10720000823089F48091D8058F5F8093D8050FE193
:1072100010E02CE330E046EE50E069E670E081E0FB
:1072200090E00E94A40480913806833089F4809114
:10723000D80581508093D8050FE110E02CE330E0B1
:1072400046EE50E069E670E081E090E00E94A40420
:107250008091D805823010F01092D8058091D80521
:1072600090E09093FA058093F90576C18091D80556
:10727000811103C01092690678C1813009F075C18F
:107280003DE6E32E33E0F32E01E02FE130E04FEF57
:107290005FEF62E370E08FE090E00E94990545EBBC
:1072A000E42E42E0F42E2FE130E04FEF5FEF66E492
:1072B00070E08FE090E00E949905E090FB05F0906F
:1072C000FC0503E02FE130E040E058EF62E870E0B9
:1072D00080E590E00E94DF058091FB059091FC0520
:1072E00090936806809367060E94DD0C80913806B3
:1072F0008230A9F480916706909168060196909378
:107300006806809367060FE110E02CE330E046EE5C
:1073100050E069E670E081E090E00E94A404809172
:1073200038068330A9F4809167069091680601972A
:1073300090936806809367060FE110E02CE330E03D
:1073400046EE50E069E670E081E090E00E94A4041F
:1073500080916706909168068B3F910520F010920E
:107360006806109267068091670690916806909370
:10737000FC058093FB05F0C08091D805882309F4B3
:1073800079CF813009F0F1C09EE9E92E92E0F92E23
:1073900001E02FE130E04FEF5FEF62E370E08FE05C
:1073A00090E00E9499052BE8E22E22E0F22E2FE1D8
:1073B00030E04FEF5FEF66E470E08FE090E00E9416
:1073C0009905E090FD05F090FE0503E02FE130E027
:1073D00040E058EF62E870E080E590E00E94DF0551
:1073E0008091FD059091FE0590934306809342069F
:1073F0000E94DD0C809138068230A9F4809142060B
:1074000090914306019690934306809342060FE1C4
:1074100010E02CE330E046EE50E069E670E081E0F9
:1074200090E00E94A404809138068330A9F48091F2
:10743000420690914306019790934306809342063B
:107440000FE110E02CE330E046EE50E069E670E03A
:1074500081E090E00E94A40480914206909143064E
:10746000C39720F010924306109242068091420684
:10747000909143069093FE058093FD056DC08EE4C8
:10748000E82E82E0F82E01E02FE130E04FEF5FEFD1
:107490006CE370E08FE090E00E949905E0900506B3
:1074A000F090060603E02FE130E040E058EF62E89C
:1074B00070E080E590E00E94DF05809105069091E4
:1074C000060690930D0680930C060E94DD0C8091B9
:1074D00038068230A9F480910C0690910D06019631
:1074E00090930D0680930C060FE110E02CE330E042
:1074F00046EE50E069E670E081E090E00E94A4046E
:10750000809138068330A9F480910C0690910D0685
:10751000019790930D0680930C060FE110E02CE389
:1075200030E046EE50E069E670E081E090E00E94D5
:10753000A4048091E7059091E8058935924020F0F8
:10754000D0920D06C0920C0680910C0690910D060B
:1075500090930606809305068FE798E321E081501B
:1075600090402040E1F700C0000080913806813053
:1075700051F48093070610927D068FE190E00E94FF
:1075800019060E942226B092380631C9DF91CF91A8
:107590001F910F91FF90EF90DF90CF90BF900895D3
:1075A000EF92FF920F931F93CF93DF93A895809153
:1075B00045068111F5C08FE190E00E9419060E94F6
:1075C0004F0C80911B0690E090931E0680931D0641
:1075D00085E080933806C1E0D5E0809145068111B1
:1075E000DFC0A8950E94DD0C809138068230A9F496
:1075F00080911D0690911E06019690931E06809321
:107600001D060FE110E02CE330E046EE50E069E6A5
:1076100070E081E090E00E94A404809138068330FD
:10762000A9F480911D0690911E06019790931E0665
:1076300080931D060FE110E02CE330E046EE50E0B1
:1076400069E670E081E090E00E94A40480911D064C
:1076500090911E06039720F010921E0610921D06B0
:10766000A89580911D0690911E068130910589F1A3
:10767000D0F0029709F046C080E7E82E84E0F82EAB
:1076800002E02FE130E04FEF5FEF6DE770E088E25E
:1076900090E00E94990582E080931B064EE150E045
:1076A00068E671E02BC024E8E22E24E0F22E02E02E
:1076B0002FE130E04FEF5FEF6DE770E088E290E0A0
:1076C0000E94990510921B064EE150E064EA71E0B9
:1076D00015C09AE7E92E94E0F92E02E02FE130E0A0
:1076E0004FEF5FEF6DE770E088E290E00E94990550
:1076F000C0931B064EE150E066E871E089EE95E02C
:107700000E9472448091380681110FC0A895C093E1
:1077100045061092240610922306C09333068FE18B
:1077200090E00E9419060E94251F80913806813042
:1077300059F5A895809345061092240610922306C9
:10774000809333068FE190E00E94190610927D0627
:1077500080911B06813069F038F0823091F44EE15F
:1077600050E068E671E009C04EE150E064EA71E083
:1077700004C04EE150E066E871E089EE95E00E94B9
:107780007244A8950E942226D09338062FEF80E7F6
:1077900092E0215080409040E1F700C000001DCFF2
:1077A000DF91CF911F910F91FF90EF900895EF928D
:1077B000FF920F931F93CF93DF93A8958091450677
:1077C0008111F3C08FE190E00E9419060E944F0CD6
:1077D0008091220690E090931E0680931D0685E01E
:1077E00080933806C1E0D5E0809145068111DDC067
:1077F000A8950E94DD0C809138068230A9F4809112
:107800001D0690911E06019690931E0680931D06FC
:107810000FE110E02CE330E046EE50E069E670E066
:1078200081E090E00E94A404809138068330A9F49E
:1078300080911D0690911E06019790931E068093DD
:107840001D060FE110E02CE330E046EE50E069E663
:1078500070E081E090E00E94A40480911D06909168
:107860001E06039720F010921E0610921D068091AE
:107870001D0690911E068130910589F1D0F0029786
:1078800009F045C080E7E82E84E0F82E02E02FE101
:1078900030E04FEF5FEF6DE770E088E290E00E942C
:1078A000990582E0809322064EE150E06EE071E09F
:1078B0002BC024E8E22E24E0F22E02E02FE130E09B
:1078C0004FEF5FEF6DE770E088E290E00E9499056E
:1078D000109222064EE150E06AE471E015C09AE78A
:1078E000E92E94E0F92E02E02FE130E04FEF5FEF58
:1078F0006DE770E088E290E00E949905C09322064F
:107900004EE150E06CE271E089EE95E0EBD78091BA
:107910003806811110C0A895C09345061092240620
:1079200010922306C09333068FE190E00E9419065F
:10793000A8950E94251F80913806813051F5A895A1
:1079400080934506109224061092230680933306F6
:107950008FE190E00E94190610927D068091220628
:10796000813069F038F0823089F44EE150E06EE009
:1079700071E009C04EE150E06AE471E004C04EE1FC
:1079800050E06CE271E089EE95E0ACD7A8950E94DA
:107990002226D09338062FEF80E792E021508040D6
:1079A0009040E1F700C000001FCFDF91CF911F9101
:1079B0000F91FF90EF900895EF92FF920F931F9316
:1079C000CF93DF93A895809145068111F4C08FE194
:1079D00090E00E9419060E944F0C80917A0690E078
:1079E00090931E0680931D0685E080933806C1E0C3
:1079F000D5E0809145068111DEC0A8950E94DD0C7E
:107A0000809138068230A9F480911D0690911E065F
:107A1000019690931E0680931D060FE110E02CE363
:107A200030E046EE50E069E670E081E090E00E94D0
:107A3000A404809138068330A9F480911D069091AA
:107A40001E06019790931E0680931D060FE110E01D
:107A50002CE330E046EE50E069E670E081E090E033
:107A60000E94A40480911D0690911E06039720F0A9
:107A700010921E0610921D0680911D0690911E0602
:107A80008130910589F1D0F0029709F045C080E777
:107A9000E82E84E0F82E02E02FE130E04FEF5FEFB8
:107AA0006DE770E088E290E00E94990582E08093A3
:107AB0007A064EE150E064EB70E02BC024E8E22E41
:107AC00024E0F22E02E02FE130E04FEF5FEF6DE7B0
:107AD00070E088E290E00E94990510927A064EE1EB
:107AE00050E060EF70E015C09AE7E92E94E0F92EBF
:107AF00002E02FE130E04FEF5FEF6DE770E088E2EA
:107B000090E00E949905C0937A064EE150E062ED44
:107B100070E089EE95E0E6D680913806811110C0BC
:107B2000A895C09345061092240610922306C09390
:107B300033068FE190E00E941906A8950E94251F48
:107B400080913806813059F5A895809345061092AA
:107B5000240610922306809333068FE190E00E9462
:107B60001906A89510927D0680917A06813069F0F9
:107B700038F0823089F44EE150E064EB70E009C0E7
:107B80004EE150E060EF70E004C04EE150E062ED85
:107B900070E089EE95E0A6D6A8950E942226D093A3
:107BA00038062FEF80E792E0215080409040E1F7C7
:107BB00000C000001ECFDF91CF911F910F91FF9069
:107BC000EF9008950F931F938091100690911106E6
:107BD000892B09F099C080917106909172068335C6
:107BE0009105A9F581E090E090931106809310062D
:107BF0000E9480130FE110E02CE330E044E650E0F7
:107C00006BE470E08EE690E00E94A40424E230E091
:107C10004AE550E064E670E088E090E00E94A40449
:107C200024E230E04AE550E064E670E088E090E06D
:107C30000E94A40424E230E04AE550E064E670E0EB
:107C40008FED90E00E94A4040E94251FA8950E9439
:107C5000091E0E94EA19A89503E02FE130E04FEFDA
:107C60005FEF69E170E085E890E00E94FD100E94FE
:107C7000B71D0E949C1080911006909111060197EB
:107C800081F5A8950E9480130FE110E02CE330E00D
:107C900044E650E06BE470E08EE690E00E94A404BD
:107CA00024E230E04AE550E064E670E088E090E0ED
:107CB0000E94A40424E230E04AE550E064E670E06B
:107CC00088E090E00E94A40424E230E04AE550E01D
:107CD00064E670E08FED90E00E94A4040E94251FEE
:107CE000A8952FEF81EE94E0215080409040E1F77D
:107CF00000C000000E94D20E0E94E01D0E94580F9A
:107D00001F910F910C94C80F1F910F9108951F920E
:107D10000F920FB60F9211248F939F938CB190E026
:107D200090937206809371069F918F910F900FBE72
:107D30000F901F9018951F920F920FB60F9211245B
:107D40002F938F939F938091E3059091E405019683
:107D5000883E23E0920728F49093E4058093E3059E
:107D600004C01092E4051092E30580910E06811183
:107D700005C010927406109273060BC0813049F44E
:107D80008091730690917406019690937406809387
:107D9000730680912D06811105C01092E2051092A4
:107DA000E1050BC0813049F48091E1059091E20535
:107DB00001969093E2058093E1058091250681115B
:107DC00005C01092E6051092E5050BC0813049F41C
:107DD0008091E5059091E60501969093E6058093E4
:107DE000E5059F918F912F910F900FBE0F901F90DF
:107DF00018952FEF89E698E1215080409040E1F7F7
:107E000000C000008FEF8ABB81BB8093610081E0DE
:107E100084BB88EA8FBD8CE08EBD1DBC1CBC17BC2A
:107E200016BC8AE78BBD82E18ABD19BC18BC1092D2
:107E3000790010927800C0E1C7BF10BE87E683BF0B
:107E400012BE11BE81E880938B0085E080938A008A
:107E50001092890010928800109281001092800088
:107E60001092870010928600109285001092840074
:107E700010928300109282001BB888E98AB986E0CC
:107E800080939500109290008FE289B98FE181BDB7
:107E90008FE081BD6CD081E00E94B0038FE190E063
:107EA0000E94190681E090E09093110680931006DD
:107EB00010922406109223061092130610921206B6
:107EC0001092E4051092E30510922A0610922906FA
:107ED0001092E00510920F06109275061092080697
:107EE00080E590E090937206809371068091640023
:107EF0008E7F80936400809165008160809365002F
:107F00007894A49AC5BB2FEF85EA9EE0215080406B
:107F10009040E1F700C0000015BA82EB92E0F2D485
:107F2000813079F00E94291AA8950E94961DA89583
:107F300061E083EB92E0FCD4A89561E082EB92E0F3
:107F4000F7D4A8958091100690911106019721F41D
:107F5000A8950E94251FA895A89534DEF2CFC09859
:107F6000AB9AAF9A8FB9779BFECF8FB1089587E018
:107F700087BBC09AAB9AAF9A83E58DB91EB880E8EB
:107F8000EEDF80E0ECDF80E0EADF8AE18A95F1F75E
:107F900000C00895EF92FF920F931F93CF93DF934A
:107FA00000D000D0CDB7DEB77C018B01A895AB9A8D
:107FB000AF9A1C821B821A82198280EDD0DF80E08A
:107FC000CEDF8FB190E09C838B838B819C81982F37
:107FD00088279C838B8380E0C2DF2FB18B819C81BB
:107FE000822B9C838B838B819C8133E09695879534
:107FF0003A95E1F79C838B8387EC90E00197F1F74A
:1080000000C0000080E9ABDF80E0A9DF8FB190E025
:108010009A83898389819A81982F88279A83898373
:1080200080E09DDF2FB189819A81822B9A83898399
:1080300089819A8153E0969587955A95E1F79A83BD
:1080400089838B819C81F7019183808389819A81C7
:10805000F801918380830F900F900F900F90DF9124
:10806000CF911F910F91FF90EF90089570D088F0FD
:108070009F5790F0B92F9927B751A0F0D1F0660F14
:10808000771F881F991F1AF0BA95C9F712C0B1302F
:1080900081F077D0B1E0089574C0672F782F8827DA
:1080A000B85F39F0B93FCCF3869577956795B3956E
:1080B000D9F73EF490958095709561957F4F8F4FDD
:1080C0009F4F0895E89409C097FB3EF490958095E2
:1080D000709561957F4F8F4F9F4F9923A9F0F92F8E
:1080E00096E9BB279395F695879577956795B7950C
:1080F000F111F8CFFAF4BB0F11F460FF1BC06F5FF2
:108100007F4F8F4F9F4F16C0882311F096E911C003
:10811000772321F09EE8872F762F05C0662371F024
:1081200096E8862F70E060E02AF09A95660F771F38
:10813000881FDAF7880F9695879597F9089557FD68
:108140009058440F551F59F05F3F71F04795880FC5
:1081500097FB991F61F09F3F79F08795089512165C
:1081600013061406551FF2CF4695F1DF08C0161608
:1081700017061806991FF1CF8695710561050894B9
:108180000895E894BB2766277727CB0197F90895D0
:108190000BD078C069D028F06ED018F0952309F084
:1081A0005AC05FC01124EECFCADFA0F3959FD1F370
:1081B000950F50E0551F629FF001729FBB27F00D95
:1081C000B11D639FAA27F00DB11DAA1F649F6627EA
:1081D000B00DA11D661F829F2227B00DA11D621F39
:1081E000739FB00DA11D621F839FA00D611D221FF3
:1081F000749F3327A00D611D231F849F600D211DD7
:10820000822F762F6A2F11249F5750408AF0E1F079
:1082100088234AF0EE0FFF1FBB1F661F771F881FC2
:1082200091505040A9F79E3F510570F014C0AACF5D
:108230005F3FECF3983EDCF3869577956795B795AD
:10824000F795E7959F5FC1F7FE2B880F911D9695D7
:10825000879597F9089597F99F6780E870E060E047
:1082600008959FEF80EC089500240A9416161706CF
:1082700018060906089500240A9412161306140617
:1082800005060895092E0394000C11F4882352F07A
:10829000BB0F40F4BF2B11F460FF04C06F5F7F4F32
:1082A0008F4F9F4F0895AA1BBB1B51E107C0AA1F08
:1082B000BB1FA617B70710F0A61BB70B881F991F87
:1082C0005A95A9F780959095BC01CD010895EE0FC0
:1082D000FF1F0024001C0BBE0790F691E02D0994AF
:1082E000A29FB001B39FC001A39F700D811D1124F7
:1082F000911DB29F700D811D1124911D0895BB2702
:108300004A3031F4992322F4BDE2909581959F4F34
:1083100001C0BB27FB015527AA27880F991FAA1F59
:10832000A41710F0A41B83955051B9F7A05DAA3390
:1083300008F0A95DA193009779F7B111B19311925B
:10834000CB0126C2CF93DF93CDB7DEB7AE014B5F33
:108350005F4FFA0161917191AF0180918006909118
:10836000810603D0DF91CF9108952F923F924F92D3
:108370005F926F927F928F929F92AF92BF92CF92B5
:10838000DF92EF92FF920F931F93CF93DF93CDB7BE
:10839000DEB72B970FB6F894DEBF0FBECDBF6C01D2
:1083A0007B018A01FC0117821682838181FFBFC194
:1083B000CE0101963C01F6019381F70193FD859171
:1083C00093FF81917F01882309F4ADC1853239F48F
:1083D00093FD859193FF81917F01853221F4B60150
:1083E00090E0E6D1E8CF912C212C312CFFE1F31560
:1083F000D8F08B3279F038F4803279F08332A1F4FE
:10840000232D20611DC08D3261F0803369F4232D4E
:10841000216016C0832D8260382EE32DE4603E2E4D
:108420002AC0F32DF8601DC037FC2DC020ED280FA9
:108430002A3040F08E32B9F436FC75C1232D206409
:10844000322E19C036FE06C08AE0989E200D1124F7
:10845000922E11C0EAE02E9E200D1124222EF32D23
:10846000F0623F2E08C08C3621F4832D8068382EB0
:1084700002C0883641F4F70193FD859193FF819105
:108480007F018111B3CF982F9F7D9554933028F4AD
:108490000C5F1F4F9FE399830DC0833631F0833704
:1084A00071F0833509F055C020C0F80180818983BF
:1084B0000E5F1F4F88248394912C530112C0280112
:1084C000F2E04F0E511CF801A080B18036FE03C0CF
:1084D000692D70E002C06FEF7FEFC5014ED14C01F6
:1084E0008201F32DFF773F2E15C0280122E0420EB6
:1084F000511CF801A080B18036FE03C0692D70E0E8
:1085000002C06FEF7FEFC5012DD14C01F32DF06854
:108510003F2E820133FC19C0822D90E08816990607
:10852000A0F4B60180E290E043D12A94F5CFF501A2
:1085300037FC859137FE81915F01B60190E038D11B
:1085400021102A9421E0821A91088114910479F76C
:10855000E1C0843611F0893639F5F80137FE07C0DD
:1085600060817181828193810C5F1F4F08C060819F
:108570007181072E000C880B990B0E5F1F4FF32D96
:10858000FF763F2E97FF09C0909580957095619575
:108590007F4F8F4F9F4FF0683F2E2AE030E0A301BE
:1085A00043D1882E861844C0853731F4232D2F7E81
:1085B000B22E2AE030E025C0932D997FB92E8F3658
:1085C000C1F018F4883579F0AEC0803719F08837DB
:1085D00021F0A9C0E92FE061BE2EB4FE0DC0FB2D35
:1085E000F460BF2E09C034FE0AC0292F2660B22EC7
:1085F00006C028E030E005C020E130E002C020E104
:1086000032E0F801B7FE07C06081718182819381F9
:108610000C5F1F4F06C06081718180E090E00E5FAB
:108620001F4FA30101D1882E8618FB2DFF773F2E07
:1086300036FE0DC0232D2E7FA22E891458F434FE51
:108640000BC032FC09C0832D8E7EA82E05C0B82C2D
:10865000A32C03C0B82C01C0B92CA4FE0FC0FE018E
:10866000E80DF11D8081803321F49A2D997EA92E89
:1086700009C0A2FE06C0B394B39404C08A2D8678C4
:1086800009F0B394A3FC10C0A0FE06C0B21480F49D
:10869000280C922C9B180DC0B21458F4B60180E23D
:1086A00090E086D0B394F8CFB21418F42B1802C01F
:1086B000982C212CA4FE0FC0B60180E390E078D066
:1086C000A2FE16C0A1FC03C088E790E002C088E5C6
:1086D00090E0B6010CC08A2D867851F0A1FE02C050
:1086E0008BE201C080E2A7FC8DE2B60190E060D091
:1086F000891430F4B60180E390E05AD09A94F8CF10
:108700008A94F301E80DF11D8081B60190E050D00C
:108710008110F6CF222009F44ECEB60180E290E01F
:1087200047D02A94F7CFF6018681978102C08FEF58
:108730009FEF2B960FB6F894DEBF0FBECDBFDF9133
:10874000CF911F910F91FF90EF90DF90CF90BF904E
:10875000AF909F908F907F906F905F904F903F90E1
:108760002F900895FC010590615070400110D8F7DA
:10877000809590958E0F9F1F0895FC016150704069
:1087800001900110D8F7809590958E0F9F1F089546
:10879000DC01FC01672F71917723E1F7329704C068
:1087A0007C916D9370836291AE17BF07C8F30895F3
:1087B0000F931F93CF93DF93FB01238121FD03C010
:1087C0008FEF9FEF2CC022FF16C046815781248176
:1087D00035814217530744F4A081B1819D012F5F79
:1087E0003F4F318320838C93268137812F5F3F4F0A
:1087F0003783268314C08B01EC01FB010084F185D3
:10880000E02D0995892BE1F6D80116968D919C9162
:108810001797019617969C938E931697CE01DF912A
:10882000CF911F910F910895FA01AA27283051F195
:10883000203181F1E8946F936E7F6E5F7F4F8F4F91
:108840009F4FAF4FB1E03ED0B4E03CD0670F781FF0
:10885000891F9A1FA11D680F791F8A1F911DA11DD5
:108860006A0F711D811D911DA11D20D009F468940E
:108870003F912AE0269F11243019305D3193DEF6B6
:10888000CF010895462F4770405D4193B3E00FD06C
:10889000C9F7F6CF462F4F70405D4A3318F0495D57
:1088A00031FD4052419302D0A9F7EACFB4E0A6953A
:1088B0009795879577956795BA95C9F7009761055C
:1088C000710508959B01AC010A2E069457954795B2
:1088D00037952795BA95C9F7620F731F841F951FA7
:1088E000A01D0895DC01CB01FC01E199FECF06C07B
:1088F000FFBBEEBBE09A31960DB20D924150504055
:10890000B8F70895E199FECF9FBB8EBBE09A9927F7
:108910008DB30895A8E1B0E042E050E0E5CFDC017E
:10892000CB0102C02D9105D041505040D8F7089599
:10893000262FE199FECF9FBB8EBB2DBB0FB6F894BF
:10894000E29AE19A0FBE01960895F2DF272FF1CF48
:04895000F894FFCFC9
:108954000000000200000000DE0700000000575481
:108964003D2025750A47530047533D2025750A537A
:108974004E00534E3D2025750A454E4400574B3D4D
:108984002025750A565000503D332E360A520052A7
:108994004C3D2025750A68004F3D73740A53004707
:1089A4003D73740A530053523D53746174696F6E7E
:1089B400200A57500057503D536E36332F506233C0
:1089C400370A57540057503D536E41670A575400B5
:1089D40057503D50726F66696C65300A57540057A2
:1089E400503D50726F66696C65310A575400575098
:1089F4003D50726F66696C65320A57540057503D9A
:108A040050726F66696C65330A57540057503D5075
:108A1400726F66696C65340A57540057503D507242
:108A24006F66696C65350A57540053523D5550685A
:108A34006561746572200A57500053523D50726547
:108A4400686561746572200A57500053523D4D6148
:108A54006E75616C200A57500053523D5265626F27
:108A64006C6C696E67200A57500053523D43686925
:108A74007068656174696E67200A57500053523DEF
:108A840050434268656174696E67200A5750005309
:108A9400523D5043200A57500056312E32002020B8
:108AA40020C2F0E5ECFF20F0E5E1EEEBEBE8EDE3CE
:108AB400E02020202000C2FBE1E5F0E8F2E520F010
:108AC400E5E6E8EC00D2E5ECEFE5F0E0F2F3F0E007
:108AD40020EFEEEBEEF7EAE8202000EDE8E7E020F7
:108AE400EFF0E820E4EEEDE0E3F0E5E2E500D2E5C6
:108AF400ECEFE5F0E0F2F3F0E020F3E2E5EBE8F789
:108B0400E5EDE8FF00202020202020E4EEEDE0E366
:108B1400F0E5E2E020202020202000C4EBE8F2E58C
:108B2400EBFCEDEEF1F2FC20E2EFE8F2FBE2E0ED2B
:108B3400E8FF00D4F3EDEAF6E8FF20E4EEEDEEE31F
:108B4400F0E5E2E000EDE8E6EDE5E3EE20EDE0E35C
:108B5400F0E5E2E0F2E5EBFF2020202000CCE0EAA3
:108B6400F1E8ECE0EBFCEDE0FF20ECEEF9EDEEF1EA
:108B7400F2FC202000E2E5F0F5EDE5E3EE20EDE087
:108B8400E3F0E5E2E0F2E5EBFF20202000CCE0EAB0
:108B9400F1E8ECE0EBFCEDE0FF20ECEEF9EDEEF1BA
:108BA400F2FC202000E2E5F0F5EDE5E3EE20EDE057
:108BB400E3F0E5E2E0F2E5EBFF20202000D2E5EC73
:108BC400EFE5F0E0F2F3F0E020E2EAEBFEF7E5EDAA
:108BD400E8FF202000CAEEEDF2F0EEEBFC20EFEE11
:108BE40020E2E5F0F5F320202020202000EDE8E647
:108BF400EDE5E3EE20EDE0E3F0E5E2E0F2E5EBFFA6
:108C04002020202000CAEEFDF4F4E8F6E8E5EDF2B9
:108C140020EFF0EEF4E8EBFF2020202000E2E5F066
:108C2400F5EDE5E3EE20EDE0E3F0E5E2E0F2E5EB7F
:108C3400FF20202000CAEEFDF4F4E8F6E8E5EDF2AA
:108C440020EFF0EEF4E8EBFF2020202000EDE0E33D
:108C5400F0E5E2E0F2E5EBFF202000D2E5ECEFE501
:108C6400F0E0F2F3F0E020EDE8E6EDE5E3EE2020BD
:108C7400202000EFE0E9EAE82000D2E5ECEFE5F09F
:108C8400E0F2F3F0E020ECE5F1F2E02020202020F7
:108C940000C2FBE1E5F0E8F2E520EFF0EEF4E8EBEA
:108CA400FC00CFF0EEF4E8EBFC203500CFF0EEF45E
:108CB400E8EBFC203400CFF0EEF4E8EBFC203300CA
:108CC400CFF0EEF4E8EBFC203200CFF0EEF4E8EB6A
:108CD400FC203100CFF0EEF4E8EBFC203000536EC2
:108CE400416700536E506200CAEEECEFFCFEF2E501
:108CF400F000C4EEEF2E20EDE0F1F2F0EEE9EAE848
:108D040000EFEBE0F20020D1F3F8EAE020EFEBE033
:108D1400F22000ECE8EAF0EEF1F5E5EC00D1F3F82E
:108D2400EAE000D0E5E1EEEBEBE8EDE32000D0F380
:108D3400F7EDEEE9002020D0F3F7EDEEE920202056
:108D440000CDE8E6EDE8E920EDE0E3F02E2000C2F6
:108D5400E5F0F5EDE8E920EDE0E3F02E002020D188
:108D6400F2E0EDF6E8FF00E2E5F0F5E000EDE8E71B
:108D7400E000CCEEF9EDEEF1F2FC00CFF0E8EDFF0F
:108D8400F2EE202000C2DBC1D0C0D2DC00C2DBCABC
:108D9400CB00C2CACB00CDE0F1F2F0EEE8F2FC0069
:108DA400C7E2F3EAEEE2FBE520F1E8E3EDE0EBFBFA
:108DB40000CFF0E5E4F3F1F2E0EDEEE2EAE800D30F
:108DC400ECEEEBF7E0EDE8FF00C2F0E5ECFF20EF9E
:108DD400E0E9EAE80020C4E0F2F7E8EA20EDE8E69A
:108DE4002E20EDE0E3F0E5E2E0F2E5EBFF0020C445
:108DF400E0F2F7E8EA20ECE5F1F2E020EFE0E9EA5E
:108E0400E800F0F3F7EDEEE900EDE8E6EDE8E9005F
:108E1400EDE0E3F02E00C2E5F0F5EDE8E900C2DB99
:048E2400D5CEC400E3
:00000001FF
